:020000040800F2
:1000000000C00020C17100080572000805720008D8
:100010000572000805720008057200080000000063
:100020000000000000000000000000000572000851
:100030000572000800000000057200080D050008A8
:1000400005720008057200080572000805720008B4
:1000500005720008057200080572000805720008A4
:100060000572000805720008057200080572000894
:100070000572000805720008057200080572000884
:100080000572000805720008057200080572000874
:100090000572000805720008057200080572000864
:1000A0000572000805720008057200080572000854
:1000B0000572000805720008057200080572000844
:1000C0000572000805720008057200080572000834
:1000D0000572000805720008057200080572000824
:1000E0000572000805720008057200080000000093
:1000F0000000000000000000000000000000000000
:1001000000000000000000000572000805720008F1
:1001100005720008057200080572000805720008E3
:1001200005720008057200080572000805720008D3
:1001300005720008057200080572000805720008C3
:1001400005720008057200080572000805720008B3
:10015000000000000000000000000000000000009F
:10016000000000000000000000000000000000008F
:10017000000000000000000000000000000000007F
:10018000000000000000000000000000000000006F
:10019000000000000000000000000000000000005F
:1001A000000000000000000000000000000000004F
:1001B000000000000000000000000000000000003F
:1001C000000000000000000000000000000000002F
:1001D000000000000000000000000000000000001F
:0401E0005FF8E0F1F3
:1001E80040F20453C2F200031A780AB901201870C9
:1001F800704700BF40F20450C2F2000008B503681F
:100208002BB140F20003C0F2000303B1984708BDC8
:1002180041F20003C4F2020310B41868194640F012
:1002280001021A600C6841F2000314F0020FC4F2D4
:100238000203F7D05C68194624F0030058605A6836
:100248005A604A6841F2000312F00C0FC4F202032C
:10025800F7D1996940F6004241F008009861C4F26C
:10026800010214684EF2100024F070411160146805
:10027800CEF2000044F080511160546842F2080C3C
:1002880024F00F015160546840F6000144F0805496
:1002980044F0010454600268C4F2010142F0030210
:1002A80002604FF47A724260986943F6000240F0A7
:1002B800040098614868C4F2010220F0F000486028
:1002C800486840F0A0004860996941F4804040F2D5
:1002D80041319861A2F80CC0118162B610BC704718
:1002E80043F60003C4F20103198843F6000211F033
:1002F800800FC4F20102F7D09080704743F60003E4
:10030800C4F20103198843F6000211F0800FC4F209
:100318000102F7D048F21F5CC5F2EB1CACFB0013DE
:1003280064215B0901FB130030339380C0B211884C
:1003380043F6000311F0800FC4F20103F7D04CF626
:10034800CD4CCCF6CC4CACFB0012D20830329A80A3
:10035800198843F6000211F0800FC4F20102F7D0A9
:100368004CF6CD4CCCF6CC4CACFB0013D90801EBC9
:100378008103A0EB43013031C8B29080704700BFC1
:1003880043F60003C4F20103198843F6000211F092
:10039800800FC4F20102F7D041F2597CCDF2B71CAC
:1003A800ACFB001342F2107C5B0B0CFB13003033E8
:1003B800938080B2118843F6000311F0800FC4F2D5
:1003C8000103F7D044F6D35CC1F2620CACFB001217
:1003D8004FF47A7C92090CFB120030329A8080B27A
:1003E80019460A8843F6000312F0800FC4F201038D
:1003F800F7D048F21F5CC5F2EB1CACFB001264217D
:10040800520901FB12003032D1B2998080B21946EC
:100418000A8843F6000312F0800FC4F20103F7D0F4
:100428004CF6CD4CCCF6CC4CACFB0012D20830329A
:10043800D1B29980198843F6000211F0800FC4F2F6
:100448000102F7D04CF6CD4CCCF6CC4CACFB0013EB
:10045800D90801EB810CA0EB4C003030C3B293807B
:10046800704700BF0309092B43F600018CBF03F155
:10047800370C03F1300CC4F201010A8843F600037B
:1004880012F0800FC4F20103F7D000F00F00092822
:10049800A3F804C00FD9373043F60001C4F20101B4
:1004A800B1F800C043F600031CF0800FC4F201034A
:1004B800F6D0988070473030EEE700BF10B504469C
:1004C800000AFFF7CFFFE0B2BDE81040CAE700BF5F
:1004D80010B50446000CFFF7F1FFA0B2BDE81040CC
:1004E800ECE700BF017861B143F60002C4F20102F3
:1004F800138813F0800FFBD0918010F8011F00299A
:10050800F6D1704740F20553C2F200031878421C36
:10051800D2B2172A1A7098BF99781AD95A78002136
:1005280019702ABB9978481CC1B2182999702BD028
:1005380008290ED11020987048F29C1248F2A01396
:10054800C4F22122C4F22123002001211060196085
:1005580070479142F0D848F29C1248F2A013C4F2B6
:100568002122C4F221230120002110601960704764
:100578009A78511ECAB29A700AB95A70EBE7102AD3
:10058800DAD10C209870D7E701225A70D4E700BF5F
:100598002DE9F04F48F29C1148F2A0120020C4F255
:1005A800212243F60003C4F221210860C4F20103AA
:1005B8001060814ABBB0184612F8011C39B1B3F873
:1005C80000C01CF0800FFAD081800132F4E743F6B6
:1005D80000040125C4F2010446F2676706952B461C
:1005E800C6F2666721AE0DF1200925464FF0000AD4
:1005F8004FF0000BCDE904ABCDE902AB07974FF004
:1006080000081F46384600F03DFA02460B46DDE971
:10061800040100F09DFACDE9000100F0ABFCDDE932
:10062800022300F1140A1946104606F808A000F043
:10063800DDF80B4647F274510246C0F60001484601
:1006480000F0C0FC9DF820206AB14946DDE902AB04
:10065800238813F0800FFBD0A28011F8012F002A05
:10066800F6D1CDE902AB08F10108B8F1400F11D07D
:100678004FA3D3E90023DDE9020100F0B7F80246F1
:100688000B46CDE9020100F0B1F805F0F3FACDE927
:100698000401B7E7079F4FF0000CCCF128000121B7
:1006A800002216F802801FFA82FE80450FD0BCF1A6
:1006B800140F59D0BEF1000F1BD1B4F8008018F008
:1006C800800FFAD04FF07C0EA5F804E00DE0B4F8E6
:1006D80000B01BF0800FFAD04FF02A0EA5F804E006
:1006E8000FFA81FABAF13F0F10DC0131013289B2F9
:1006F800D7E7B4F800B01BF0800FFAD00FFA81FAF0
:100708004FF02003BAF13F0FAB80EEDD208810F0E8
:10071800800FFBD04FF00D02AA80218811F0800FC6
:10072800FBD00CF1010C4FF00A08BCF1290FA5F819
:100738000480B2D147F28452C0F600026421B4F8B2
:1007480000C01CF0800FFAD0A18012F8011F002908
:10075800F5D1069A501C83B206931BB2142B7FF76F
:1007680045AF0123069341E70FFA8EFB87FB0BA8E1
:100778004FEAEB7ACAEBA80303EB8308ABEB480A12
:100788000FFA8AF34BB9B4F800E01EF0800FFAD0E4
:100798004FF07C0BA5F804B0A2E7238813F0800F74
:1007A800FBD04FF02D0AA5F804A099E7AFF300801D
:1007B8001A271792BF15B03F61750008AFF3008084
:1007C80040F20852C2F20002136840F24451002B72
:1007D800C2F2000108BF0B4618181060184670478F
:1007E80081F0004102E000BF83F0004330B54FEADA
:1007F80041044FEA430594EA050F08BF90EA020F47
:100808001FBF54EA000C55EA020C7FEA645C7FEAD9
:10081800655C00F0E2804FEA5454D4EB5555B8BFFC
:100828006D420CDD2C4480EA020281EA030382EA6D
:10083800000083EA010180EA020281EA0303362DFF
:1008480088BF30BD11F0004F4FEA01314FF4801CD2
:100858004CEA113102D0404261EB410113F0004FE4
:100868004FEA03334CEA133302D0524263EB43039B
:1008780094EA050F00F0A780A4F10104D5F1200E39
:100888000DDB02FA0EFC22FA05F2801841F1000194
:1008980003FA0EF2801843FA05F359410EE0A5F168
:1008A80020050EF1200E012A03FA0EFC28BF4CF099
:1008B800020C43FA05F3C01851EBE37101F000454F
:1008C80007D54FF0000EDCF1000C7EEB00006EEB5C
:1008D8000101B1F5801F1BD3B1F5001F0CD34908E6
:1008E8005FEA30004FEA3C0C04F101044FEA44523D
:1008F80012F5800F80F09A80BCF1004F08BF5FEAC4
:10090800500C50F1000041EB045141EA050130BDA3
:100918005FEA4C0C404141EB010111F4801FA4F146
:100928000104E9D191F0000F04BF01460020B1FA9B
:1009380081F308BF2033A3F10B03B3F120020CDAD3
:100948000C3208DD02F1140CC2F10C0201FA0CF0B1
:1009580021FA02F10CE002F11402D8BFC2F1200C16
:1009680001FA02F120FA0CFCDCBF41EA0C019040CC
:10097800E41AA2BF01EB0451294330BD6FEA040415
:100988001F3C1CDA0C340EDC04F11404C4F1200200
:1009980020FA04F001FA02F340EA030021FA04F312
:1009A80045EA030130BDC4F10C04C4F1200220FA69
:1009B80002F001FA04F340EA0300294630BD21FAA7
:1009C80004F0294630BD94F0000F83F4801306BF6D
:1009D80081F480110134013D4EE77FEA645C18BF61
:1009E8007FEA655C29D094EA050F08BF90EA020FF8
:1009F80005D054EA000C04BF1946104630BD91EAF0
:100A0800030F1EBF0021002030BD5FEA545C05D1F2
:100A18004000494128BF41F0004130BD14F5800431
:100A28003CBF01F5801130BD01F0004545F0FE41A5
:100A380041F470014FF0000030BD7FEA645C1ABFDA
:100A4800194610467FEA655C1CBF0B46024650EA11
:100A5800013406BF52EA033591EA030F41F400213D
:100A680030BD00BF90F0000F04BF0021704730B5C3
:100A78004FF4806404F132044FF000054FF0000198
:100A880050E700BF90F0000F04BF0021704730B559
:100A98004FF4806404F1320410F0004548BF40422E
:100AA8004FF000013EE700BF42004FEAE2014FEA83
:100AB80031014FEA02701FBF12F07F4393F07F4F5E
:100AC80081F06051704792F0000F14BF93F07F4F90
:100AD800704730B54FF4607401F0004521F00041D3
:100AE80020E700BF50EA010208BF704730B54FF059
:100AF80000050AE050EA010208BF704730B511F05E
:100B0800004502D5404261EB41014FF4806404F195
:100B180032045FEA915C3FF4DCAE4FF003025FEA17
:100B2800DC0C18BF03325FEADC0C18BF033202EB9F
:100B3800DC02C2F1200300FA03FC20FA02F001FAF9
:100B480003FE40EA0E0021FA02F11444C1E600BF98
:100B580070B54FF0FF0C4CF4E06C1CEA11541DBF4B
:100B68001CEA135594EA0C0F95EA0C0F00F0DEF816
:100B78002C4481EA030621EA4C5123EA4C5350EAFB
:100B8800013518BF52EA033541F4801143F480134C
:100B980038D0A0FB02CE4FF00005E1FB02E506F0DD
:100BA8000042E0FB03E54FF00006E1FB03569CF032
:100BB800000F18BF4EF0010EA4F1FF04B6F5007F38
:100BC80064F5407404D25FEA4E0E6D4146EB0606AA
:100BD80042EAC62141EA55514FEAC52040EA5E5033
:100BE8004FEACE2EB4F1FD0C88BFBCF5E06F1ED8DD
:100BF800BEF1004F08BF5FEA500E50F1000041EB14
:100C0800045170BD06F0004646EA010140EA0200C0
:100C180081EA0301B4EB5C04C2BFD4EB0C0541EAE2
:100C2800045170BD41F480114FF0000E013C00F3F7
:100C3800AB8014F1360FDEBF002001F0004170BD1B
:100C4800C4F10004203C35DA0C341BDC04F1140434
:100C5800C4F1200500FA05F320FA04F001FA05F2C0
:100C680040EA020001F0004221F0004110EBD3708D
:100C780021FA04F642EB06015EEA430E08BF20EAB9
:100C8800D37070BDC4F10C04C4F1200500FA04F35C
:100C980020FA05F001FA04F240EA020001F00041EE
:100CA80010EBD37041F100015EEA430E08BF20EA61
:100CB800D37070BDC4F1200500FA05F24EEA020EA9
:100CC80020FA04F301FA05F243EA020321FA04F0D8
:100CD80001F0004121FA04F220EA020000EBD3708F
:100CE8005EEA430E08BF20EAD37070BD94F0000F8F
:100CF8000FD101F00046400041EB010111F4801FC3
:100D080008BF013CF7D041EA060195F0000F18BF73
:100D1800704703F00046520043EB030313F4801FAF
:100D280008BF013DF7D043EA0603704794EA0C0F69
:100D38000CEA135518BF95EA0C0F0CD050EA41067F
:100D480018BF52EA4306D1D181EA030101F00041FC
:100D58004FF0000070BD50EA410606BF1046194624
:100D680052EA430619D094EA0C0F02D150EA013630
:100D780013D195EA0C0F05D152EA03361CBF104671
:100D880019460AD181EA030101F0004141F0FE4110
:100D980041F470014FF0000070BD41F0FE4141F494
:100DA800780170BD70B54FF0FF0C4CF4E06C1CEA94
:100DB80011541DBF1CEA135594EA0C0F95EA0C0F49
:100DC80000F0A7F8A4EB050481EA030E52EA033504
:100DD8004FEA013100F088804FEA03334FF0805525
:100DE80045EA131343EA12634FEA022245EA111552
:100DF80045EA10654FEA00260EF000419D4208BF03
:100E0800964244F1FD0404F5407402D25B084FEAAF
:100E18003202B61A65EB03055B084FEA32024FF45B
:100E280080104FF4002CB6EB020E75EB030E22BFB8
:100E3800B61A754640EA0C005B084FEA3202B6EB78
:100E4800020E75EB030E22BFB61A754640EA5C0027
:100E58005B084FEA3202B6EB020E75EB030E22BFB7
:100E6800B61A754640EA9C005B084FEA3202B6EBB8
:100E7800020E75EB030E22BFB61A754640EADC0077
:100E880055EA060E18D04FEA051545EA16754FEAD9
:100E980006164FEAC30343EA52734FEAC2025FEAF7
:100EA8001C1CC0D111F4801F0BD141EA00014FF086
:100EB80000004FF0004CB6E711F4801F04BF014357
:100EC8000020B4F1FD0C88BFBCF5E06F3FF6AFAE73
:100ED800B5EB030C04BFB6EB020C5FEA500C50F103
:100EE800000041EB045170BD0EF0004E4EEA113186
:100EF80014EB5C04C2BFD4EB0C0541EA045170BD8D
:100F080041F480114FF0000E013C90E645EA060ED0
:100F18008DE60CEA135594EA0C0F08BF95EA0C0FFE
:100F28003FF43BAF94EA0C0F0AD150EA01347FF446
:100F380034AF95EA0C0F7FF425AF104619462CE71D
:100F480095EA0C0F06D152EA03353FF4FDAE104680
:100F5800194622E750EA410618BF52EA43067FF4D1
:100F6800C5AE50EA41047FF40DAF52EA43057FF461
:100F7800EBAE12E74FEA410212F5001215D211D575
:100F88006FF47873B3EB625212D94FEAC12343F07E
:100F9800004343EA505311F0004F23FA02F018BF00
:100FA800404270474FF00000704750EA013005D1C9
:100FB80011F0004008BF6FF0004070474FF000008C
:100FC800704700BF0EB440F2000330B59CB01FACB0
:100FD800C2F20003054601A954F8042B4FF0FF3C68
:100FE80018684FF40273ADF8103023460595019543
:100FF8006FF00045ADF812C0069503951B9400F0FC
:10100800B9F8019B00221A701CB0BDE8304003B04B
:10101800704700BF0CB40B4610B59CB01EAC01A9BC
:1010280005934FF4027C54F8042B01934FF0FF33DF
:10103800ADF8123023461B946FF00044ADF810C091
:101048000694039400F096F8019B00221A701CB0D5
:10105800BDE8104002B070472DE9F04F85B09246C8
:101068000C46039090681768002800F081804FF0C4
:1010780000090B684D46002D54D0A668B542B0460D
:101088003EBF18462E46A8463CD3A08910F4906F60
:1010980008BF184636D06269216902EB420B5B1A19
:1010A80003F1010C0BEBDB7BAC444FEA6B0BE34524
:1010B8005A463CBFE3465A4610F4806F37D0114673
:1010C8000398019302F0F6FB019B00283BD01A46D7
:1010D80021690193029002F0F9FEA289019BDDF8D3
:1010E80008C022F4906242F08002A2812E46A846EF
:1010F800C3EB0B020CEB0300A260C4F810C0206025
:10110800C4F814B04246494602F0A8FFA268236812
:10111800961BA660DAF8082043442360551BCAF8DA
:101128000850FDB1D7F800907D680837A3E7039809
:10113800019303F09FFC019B84460028D6D10398B5
:10114800216902F08DFA039A0C234FF0FF301360E7
:101158000023A289CAF8043042F04002CAF80830D5
:10116800A28102E02846CAF8045005B0BDE8F08F15
:101178005060FAE72DE9F04FC5B00E469A4615467D
:10118800099002F053FBB38913F0800F00681B909D
:1011980003D03369002B01F08C800DF17409B3463C
:1011A8004C46002210920023189217921A920D9220
:1011B8002DAA199328320DF1F703169207930023ED
:1011C800CDF8DC90389339932B78B3F1250218BF0A
:1011D8000122002B0CBF002202F0010202B32E46AE
:1011E80016F8013F1A1E18BF0122252B0CBF00223A
:1011F80002F00102002AF3D1771B08BF35460FD051
:101208006760389B399A01332560D219072B3992C8
:10121800389379DC08340D983546C0190D90337829
:10122800002B00F0378700214FF00002CDF828A0EE
:101238006B1C0C914FF0FF388DF80F218A466A78A5
:101248002B204FF0200C5D1CA2F12003582B00F23C
:101258001982DFE813F02902170217023502170274
:10126800170217021702170217023C024802170258
:10127800C802CF021702EF02F602F602F602F602E1
:10128800F602F602F602F602F60217021702170233
:1012980017021702170217021702170217024F0246
:1012A8008802170288021702170217021702C102E2
:1012B80017021702EE031702170217021702170286
:1012C800930317021702AD0317021702170217023A
:1012D800170217021702170217021702C703D803CB
:1012E8008802880288020B03D803170217020F032B
:1012F8001702190329033E038C0317025903170227
:10130800840317021702EA000998594637AAFFF71B
:10131800A3FE00287CD14C467DE71899012940F3AB
:101328005284119A01236360389B2260399A0133F1
:1013380038930132072B399200F39685083401233C
:101348006360389B399A01331B980132072B399215
:101358002060389300F37D8508341098002200231C
:10136800199904F0E1F8002840F003851899119BB9
:101378004A1E6260591C389B2160399901333893A1
:101388008A18072B399200F32F8408341A9A1A986E
:1013980062603EAA389B2260399A0133389312184A
:1013A800072B399200F34F8104F108031AF0040F58
:1013B80000F056810C990B9A8E1A002E40F350813A
:1013C800102E47F20827D8BFC0F6000740F3DE8387
:1013D8001024C0F600070DF1DC08DDF824A003E0B6
:1013E800103E102E40F3D2835C60389A399901324E
:1013F8001F601031072A399103F108033892EFDD95
:10140800504659464246FFF727FE4B460028E7D08C
:101418005E46B3890D9813F0400F18BF4FF0FF30A8
:101428000D900D9845B0BDE8F08F1AF0200F47F2E7
:10143800B050C0F600001492179000F0C3820A99C9
:10144800CB1D23F0070303F108020A92D3E90067D2
:1014580056EA07010CBF002201221AEA020F40F0E7
:10146800BC8402234FF000018DF80F11B8F1000F72
:10147800A8BF2AF0800AB8F1000F18BF42F0010295
:10148800002A00F06081012B00F03484022B00F068
:1014980017841699CDF82C8011914FEAD6084FEA97
:1014A800D70C48EA477806F00700674646463030CA
:1014B80056EA070201F8010DEFD11AF0010FDDF825
:1014C8002C80119140F0DB84169B5B1A0E930E9BC7
:1014D800CDF854804345B8BF43460B939DF80F3170
:1014E80013B10B9901310B911AF00202139202D039
:1014F8000B9B02330B931AF08400129038D10C998D
:101508000B9A8E1A002E33DD102E47F20827D8BF0B
:10151800C0F6000720DD4FF01008C0F6000702E013
:10152800103E102E18DDC4F80480389B399A013318
:1015380027601032072B399204F108043893EFDD45
:101548000998594637AA4C46FFF786FD00287FF4CC
:101558005FAF103E102EE6DC6660389B27605A1C91
:10156800399B38929B19072A399300F3F78308347B
:101578009DF80F3173B101236360389B43AA03328E
:101588002260399A013338930132072B399200F3DC
:1015980040830834139B6BB102236360389B43AAD2
:1015A8002260399A013338930232072B399200F3BB
:1015B8003A8308341298802800F0B28215980E9B5E
:1015C800C61A002E2EDD102EA74FC8BF4FF01008E8
:1015D80003DC1BE0103E102E18DDC4F80480389B95
:1015E800399A013327601032072B399204F1080425
:1015F8003893EFDD0998594637AA4C46FFF72CFD7A
:1016080000287FF405AF103E102EE6DC6660389B9C
:1016180027605A1C399B38929B19072A399300F383
:10162800EE8208341AF4807F40F019820E99119ADC
:101638006160389B2260399A013338935218072B1E
:1016480039927FF7B1AE0998594637AAFFF704FDDA
:1016580000287FF4DDAE1AF0040F4B467FF4AAAEE3
:10166800399B0D980B9A0C998A42ACBF8018401888
:101678000D90002B40F09E820023DDF828A03893BF
:101688004C46A1E51492002A00F0048501208DF84B
:10169800B4204FF000012DAA0B908DF80F11119274
:1016A8000E90002115911FE79DF80F31002B40F097
:1016B8000C840A992B468DF80FC12A780A91C2E545
:1016C8000A994AF0010A2A782B460A91BBE50A9B37
:1016D8000A9A1B68111D002B0C93C0F2B2852A7858
:1016E8002B460A91AFE50A992B468DF80F012A7807
:1016F8000A91A8E54AF0100A14921AF0200F00F097
:1017080087810A98C31D23F0070303F108010A9192
:10171800D3E90067002E77F10000C0F2768356EA1D
:1017280007014FF001030CBF00220122B8F1000F9E
:10173800A8BF2AF0800AB8F1000F18BF42F00102D2
:10174800002A7FF4A0AE002B40F0E5811AF0010FCB
:1017580000F0E18130238DF8DB302DAB01202733F9
:101768000E901193B3E61AF0080F149200F0BF839D
:101778000A98C31D23F0070303F108010A915E6864
:101788001F68199610973846314603F04DFB0346FB
:10179800002800F09384384600220023314603F0E5
:1017A800CDFE002840F015849DF80F31032047F244
:1017B800A45247F2A0510B901498C0F60001C0F64D
:1017C80000022AF0800A4728D8BF0A46032111924E
:1017D80000220E91159283E60A994AF0080A2A789F
:1017E8002B460A912FE50A992A784AF0040A2B46D3
:1017F8000A9128E52B4613F8012B2A2A00F0CF86F8
:10180800A2F13001092988BF4FF0000810D802352D
:101818004FF0000815F8012C08EB88082B46013515
:1018280001EB4808A2F130010929F3D948EAE87820
:101838001D4609E50A994AF0800A2A782B460A913A
:1018480001E5A2F1300100262B4606EB860613F8C7
:10185800012B01EB4606A2F130011D460929F3D9F7
:101868000C961D46F0E400BF187200084AF0400AC2
:101878000A9934E72A786C2A00F018840A994AF001
:10188800100A2B460A91DEE41AF0200F00F0238399
:101898000A990D9A0B6810464FEAE0710A9AC3E953
:1018A800000102F1040A8FE41AF02003149200F0F8
:1018B800C7800A9BDA1D002322F0070202F1080004
:1018C8000A90D2E9006756EA07010CBF00220122FC
:1018D800C8E50A9A47F2B0500A997823C0F6000082
:1018E8001493166804318DF80D314AF0020A30233A
:1018F800321E18BF01228DF80C3136464FF0000712
:10190800179002230A91ADE50A9B14924FF000024A
:10191800181D8DF80F211B680A901193002B00F0F9
:101928004D85B8F1000F1198C0F22A850021424672
:1019380002F092FA0346002800F06E8511981B1AEF
:101948000E93434540F38284CDF83880002128EA7D
:10195800E8789DF80F31CDF82C801591C0E51AF084
:10196800200F149210D00A9BDA1D0123A4E70A99CC
:101978004AF0200A2A782B460A9164E44AF0100AB1
:1019880014921AF0200FEED11AF0100F40F0548282
:101998001AF0400F00F050820A980123011D0A91A5
:1019A8000688321E18BF012236464FF0000759E557
:1019B8001AF0200F149247F28C52C0F600021792C8
:1019C8007FF43DAD1AF0100F40F02D821AF0400F51
:1019D80000F029820A990A1D0A920E8836464FF0AD
:1019E800000735E5149201200A9A4FF000010B9088
:1019F8000E90136804328DF80F110A922DAA8DF8F3
:101A0800B43011924DE61AF0200F14927FF479AE9B
:101A18001AF0100F40F0ED811AF0400F00F0E98144
:101A28000A98011D0A91B0F9006036464FEAE67738
:101A380070E64AF0100A14921AF020037FF439AFC6
:101A48001AF0100200F05F820A9A101D0A901668B8
:101A5800321E18BF012236464FF0000702E5149BDC
:101A6800652B7FF75AAC109800220023199903F0D0
:101A78005BFD002800F0E18001236360389A47F29B
:101A8800CC53C0F600032360399B013238920133EE
:101A9800072A3993D8BF04F1080300F39F82429ABA
:101AA8001898824203DB1AF0010F3FF47FAC1B99B0
:101AB80001225A60389A19603999013238920131F5
:101AC800072A399100F3EB830833189A561E002E23
:101AD8007FF76CAC102EA04F40F3E98110240DF174
:101AE800DC0803E0103E102E40F3E1815C60389A78
:101AF800399901321F601031072A399103F108031F
:101B08003892EFDD099859464246FFF7A5FA4B4649
:101B18000028E7D07CE4169900220E921191D6E4B1
:101B28000C990B9A8E1A002E7FF748AD102E8A4F0B
:101B3800C8BF4FF0100803DC1BE0103E102E18DD64
:101B4800C4F80480389B399A013327601032072B78
:101B5800399204F108043893EFDD0998594637AAF9
:101B68004C46FFF779FA00287FF452AC103E102E4D
:101B7800E6DC6660389B27605A1C399B38929B19B3
:101B8800072A399300F38881083417E55E60389A8C
:101B98001F60399B01323892F318072A39937FF76F
:101BA80060AD0998594637AAFFF756FA00283FF45E
:101BB80057AD2DE40998594637AAFFF74DFA002882
:101BC8003FF45AAD24E41AF0010F7FF4AAAB0123C5
:101BD8006360389B399A013311990132072B399286
:101BE800216038937FF7D1AB0998594637AAFFF798
:101BF80033FA00287FF40CAC4C46FFF7C7BB0998B2
:101C0800594637AAFFF728FA00287FF401AC4C465A
:101C180008E50998594637AAFFF71EFA00287FF405
:101C2800F7AB4C46B6E40998594637AAFFF714FAB9
:101C380000287FF4EDAB4C46BCE4429B002B40F3FC
:101C4800D98118998B42C0F26F81119A6160389BD3
:101C58002260399A013338935218072B3992D8BF2A
:101C680004F1080300F3BA83429C1898241A002C44
:101C780040F39B81102C384F40F38B81CDF838A06E
:101C88001026AA460DF1DC08099D03E0103C102C33
:101C980040F37C815E60389A399901321F601031B7
:101CA800072A399103F108033892EFDD284659468F
:101CB8004246FFF7D1F94B460028E7D0FFF7A8BB0B
:101CC8001698DDF85CC003461190310906F00F0242
:101CD80041EA077138091CF802200E46074656EA01
:101CE800070103F8012DF0D1169A1193D21A0E921A
:101CF800FFF7EDBB00230922B24273EB0700169BE6
:101D08003EBFCDF82C80A0461C461AD23046394634
:101D18000A22002303F03AFC30463946002302F138
:101D2800300C0A2204F801CD03F030FC06460F46B9
:101D380009200021B042B941E8D323464446DDF8E2
:101D48002C805A1E3036119203F8016C169B9B1A90
:101D58000E93FFF7BCBB00BF1872000809985946DC
:101D680037AAFFF779F900287FF452AB4C46FFF702
:101D7800FFBB1898461E002E7FF708AB102E9C4F0D
:101D8800C8BF4FF0100803DC1BE0103E102E18DD12
:101D9800C4F80480389B399A013327601032072B26
:101DA800399204F108043893EFDD0998594637AAA7
:101DB8004C46FFF751F900287FF42AAB103E102E4D
:101DC800E6DC6660389B399A013327609219072B45
:101DD800399238937FF7D9AA06E7149830214AF048
:101DE800020A012202238DF80C118DF80D01FFF76C
:101DF80039BB0A9A131D16680A9336464FEAE677E6
:101E0800002E77F10000BFF68AAC764267EB4707F1
:101E18002D2356EA07028DF80F310CBF002201224C
:101E28000123FFF723BB0A9B181D1E680A9036463C
:101E38004FF00007FFF70CBB0A9A131D16680A93A8
:101E48000123321E18BF012236464FF00007FFF764
:101E580009BB0998594637AAFFF7FEF800287FF40E
:101E6800D7AA4C46FFF779BA0998594637AAFFF717
:101E7800F3F800287FF4CCAA4C46FFF760BA302864
:101E880000F09682119A302302F8013D169B1192B8
:101E98009B1A0E93FFF71BBB0998594637AAFFF701
:101EA800DBF800287FF4B4AA4C46FFF787BB5E60D6
:101EB800389A399901321F608919072A399138925D
:101EC8003FF7C1AB0833FFF771BA0A992B462A7856
:101ED8000A91FFF7B8B91AF0100F00F0CD810A98EF
:101EE8000D9900F1040A03681960FFF76DB90A9AA1
:101EF800D31D23F0070303F108000A905E681F68EA
:101F0800199610973FE41AF0400300F0A9810A9946
:101F180013460A1D0A920E88321E18BF0122364641
:101F28004FF00007FFF79EBA119A63603899226054
:101F3800399A01313891D3180729399300F362820D
:101F480008340123429E6360389B399A01331B98F9
:101F58000132072B3893D8BF04F108032060399267
:101F680000F34682429A119918988E191E60811AB8
:101F7800596039998A1A3899121839920131389169
:101F880007293FF760AB0833FFF710BA5546DDF86D
:101F980038A05C60389A399901321F600919072AFC
:101FA8003991389200F37F8208331AF0010F3FF419
:101FB800FDA91B9901225A60389A19603999013292
:101FC80038920131072A39913FF73DAB0833FFF7C3
:101FD800EDB92D238DF80F31FFF7E8BB0998594665
:101FE80037AAFFF739F800287FF412AA4B4656E5BE
:101FF8001872000801236360389A47F2CC53C0F680
:1020080000032360399B013238920133072A399340
:10201800D8BF04F1080300F37381429A2AB91898CB
:1020280018B91AF0010F3FF4C1A91B9901225A608F
:10203800389A19603999013238920131072A399151
:1020480000F368810833429C6442002C40F3878186
:10205800102C9E4F40F3A08110260DF1DC0803E000
:10206800103C102C40F398815E60389A39990132FF
:102078001F601031072A399103F108033892EFDD08
:10208800099859464246FEF7E7FF4B460028E7D035
:10209800FFF7BEB9399B5E46002B3FF4BAA90998F1
:1020A800594637AAFEF7D8FFFFF7B3B90A994AF09D
:1020B800200A6A786B1C0A91FFF7C5B83846314682
:1020C800089302F0C3FE089B002840F00181B8F194
:1020D800FF3F08BF08F107080ED0149A672A14BFFB
:1020E80000230123472A08BF43F0010323B1B8F1B5
:1020F800000F08BF4FF0010833463A46CDE93A23AE
:102108004AF4807A3B9B002BC0F20A820023159385
:102118001499662914BF00230123462908BF43F0F8
:1021280001031293002B00F08A810323CDF82C8041
:102138000B990E970F9600930998DDE90E230191EC
:1021480042A9029141A9039140A9049100F0E8FA3B
:10215800149AB2F1670318BF0123472A0CBF002362
:1021680003F0010311902BB91AF0010F08BFDDF835
:1021780000C11AD0119B0B98129903EB000C29B1DE
:102188001B78302B00F0D080429B9C4438460022BC
:1021980000233146CDF820C003F0C6F9DDF820C091
:1021A800002800F07381CDF800C1149811996728B0
:1021B80014BF00230123472808BF43F00103C1EBE4
:1021C8000C011891002B00F04A81429A12F1030F7A
:1021D8000E9202DB904580F24B81149B023B1493D4
:1021E8000E9A1498531E4293002B8DF8F800C0F2F3
:1021F800D1812B228DF8F920092B00F362813FA9A8
:1022080030338DF8FB3030238DF8FA303EAB189A16
:10221800CB1A18991A935918012A0E9140F3CC81B8
:102228000E9801300E9020EAE0710B91159B002B5F
:1022380000F0FD802D2300208DF80F311590FFF759
:1022480050B90C9B5B420C93FFF7CEBA0E9A002054
:102258009DF80F3122EAE27215900B92FFF740B910
:102268000A98011D0A910668321E18BF01223646D7
:102278004FF00007FFF7F6B81AF0400F17BF0A9A99
:102288000A990D9802F1040A11BF136801F1040AB2
:102298000B680D9A14BF18801A60FEF795BF09984D
:1022A800594637AAFEF7D8FE00287FF4B1A84B4656
:1022B8000BE40998402101F0FDFA306030610028F4
:1022C80000F08D8140237361FEF767BF1872000824
:1022D800032047F2AC5247F2A8510B901498C0F66D
:1022E8000001C0F6000215934728D8BF0A462AF015
:1022F800800A032111929DF80F310E91FFF7F0B873
:102308000998594637AAFEF7A7FE00287FF480A847
:102318004B4682E60998594637AAFEF79DFE0028E3
:102328007FF476A84B468EE63846002200233146D5
:10233800CDF820C003F0F8F8DDF820C000287FF4BD
:1023480023AF0B9AC2F1010342931EE7099859463D
:1023580037AAFEF781FE00287FF45AA84B46189A40
:1023680011985A60389A3999186001321898389239
:102378000918072A39913FF766A90833FFF716B8F5
:102388000021159102F072FE9DF80F3120EAE072EB
:102398000E900B92FFF7A4B85C60389A1F60511C2E
:1023A800399A3891121907293992CFDC0833D6E7C0
:1023B80016991198081A0E90FFF789B8B8F1060F08
:1023C80034BF4146062147F2C452C0F6000221EA52
:1023D800E1730E9111920B93FFF763B9099859466F
:1023E80037AAFEF739FE00287FF412A84B463BE4D3
:1023F8000998594637AAFEF72FFE00287FF408A847
:102408004B46AFE50998594637AAFEF725FE00283E
:102418007EF4FEAF4C4694E5CDF8388028EAE8789B
:102428001590CDF82C809DF80F31FFF759B80E980C
:102438009DF80F3120EAE0700B90FFF751B8149A1D
:10244800652A14BF00230123452A08BF43F001036E
:10245800002B32D008F101030B93022368E614988D
:10246800652862DD149A662A1CBF429B0E936FD0C2
:10247800189A0E9B9A425BDC1AF0010F40F081809B
:1024880023EAE37067210B901491CFE6409B9C45AB
:1024980098BF9C467FF689AE302203F8012B9C45F5
:1024A8004093FAD881E60998594637AAFEF7D4FD31
:1024B80000287EF4ADAF4B4677E5CDF82C8002338B
:1024C80036E646F2676C0DF1F700C6F2666C8CFBD7
:1024D8000321DA17C2EBA10202EB8201A3EB41014F
:1024E80013463031092A00F8011DF0DC3033421E52
:1024F800D9B200F8011C079B934298BF0DF1FA016D
:102508007FF684AE02460DF1FB0301E012F8011BD1
:1025180003F8011C1946079801339042F6D875E66E
:102528002D2006F100461590F2E542990E9157E6E6
:102538000E9918980029DABF0E9AC2F102030123F6
:102548001B18672123EAE3720E9314910B926DE630
:10255800429800280E9038DDB8F1000F07D11AF024
:10256800010F04BF20EAE0710B913FF45FAE0E9AB1
:1025780066201490531C43440E9323EAE3710B9195
:1025880054E60E9A6723149301320E9222EAE270FF
:102598000B904BE62D225B428DF8F9202CE60A9928
:1025A8001A78D1F8008004310A91B8F1000FB8BF49
:1025B8004FF0FF38FEF747BE1AF0010F04BF21EABB
:1025C800E1730B933FF432AE2AE6B8F1000F0ED157
:1025D8001AF0010F0BD101220B920E9226E60998F0
:1025E8000C234FF0FF310D910360FEF71ABF08F17D
:1025F8000203662023EAE3710E9314900B9115E60B
:102608002DE9F84F03690E69824689469E4200F318
:102618008380F21C01F1140500F11404013E9200BC
:102628008B18121803F1040859685068013102F038
:10263800E7FD0746002839D000239C461A46E9588A
:10264800E0581FFA81FE4FEA114B81B20EFB07CE0C
:1026580051180BFB07FC0CEB1E4C1FFA8EFECEEB41
:1026680001011FFA8CF24FEA1C4CC2EB10421FFA10
:1026780081FE02EB21424EEA0241E150043312147A
:1026880059198845DBD2321D0AEB8203596869B9AA
:102698009C4209D25AF8222012B105E01A681AB9E8
:1026A800043B013E9C42F9D3CAF8106049465046A3
:1026B80001F086FD00282CDB002301379C46EA58F0
:1026C800E05891B2120C1FFA80F9C2EB1042C1EB2C
:1026D8000901614402EB214289B241EA0241E15019
:1026E80004334FEA224C5A199045E8D2321D0AEBBE
:1026F8008203596869B99C4209D25AF8222012B15A
:1027080005E01A681AB9043B013E9C42F9D3CAF89D
:1027180010603846BDE8F88F0020BDE8F88F00BF8C
:102728002DE9F04F466AA1B00446904699462D9D82
:10273800002E00F02384326882B1616A4FF0010CE8
:10274800766820460B6856604A6819460CFA02F209
:102758009A6001F06FFE636A00221A60B9F1000600
:1027680038DB00232B6040F20003C7F6F0731A46EB
:1027780006EA0303934217D0002200234046494645
:10278800CDE9068902F0D0FE002829D02C98012333
:102798002E990360002900F0D080794B581E2E9A9C
:1027A800136021B0BDE8F08F2C9842F20F730360DC
:1027B800B8F1000F00F0958047F2DC50C0F6000039
:1027C8002E990029EDD0C278C31C002AE7D000F169
:1027D8000803E4E726F000460123B1462B60C2E770
:1027E8002046DDE906231EA900911FA9019101F0E9
:1027F80073FEC6F30A558346002D7ED0DDE9060137
:10280800A5F57E751F9F073D21F07F4323F47003D4
:1028180043F07E51002341F4E001199340F2000394
:102828000022C3F6F873FDF7DFFF4FA3D3E90023B7
:10283800FEF78EF94EA3D3E90023FDF7D7FFCDE9C4
:1028480008012846FEF71EF94BA3D3E90023FEF73B
:102858007FF902460B46DDE90801FDF7C7FFCDE920
:102868000801FEF787FB002200230646DDE9080180
:1028780002F064FE40B13046FEF704F9DDE90823B2
:1028880002F052FE00B9013E162E5BD901231893BF
:10289800013FB7EB050A42BFCAF1000ACDF83CA0D8
:1028A8004FF0000A01D400220F92002EC0F271836B
:1028B800B2440023179615932A9B092B62D8052B3F
:1028C80040F377862A98002704382A902A998B1E85
:1028D800032B00F2DD83DFE813F0A503D803D5034B
:1028E800C40326F07F4626F47006002E7FF464AFFA
:1028F80047F2D050C0F6000062E71F9F1E9BFB18EE
:1029080003F586639D1C202DDCBFC5F1200008FA65
:1029180000F008DD1E3BC5F1400216FA02F228FA63
:1029280003F342EA0300FEF79DF8A5F58665012248
:10293800033D1992A1F1F87170E747F2CC50C0F647
:1029480000002EE747F26023DDE90601C0F6000328
:1029580003EBC603D3E9002302F0F0FD002840F0A2
:102968002083189094E700BF61436F63A787D23F25
:10297800B3C8608B288AC63FFB799F501344D33F66
:10298800CD75000800234FF0FF301F4601212A9320
:102998001190169108902B93656A00236B6020466E
:1029A800696801F063FD636A28601B681093002F53
:1029B80000F05B81002E40F32A8447F2602306F082
:1029C8000F02C0F60003351103EBC20315F0100F18
:1029D800D3E90001CDE90C0100F0E78247F2383372
:1029E800DDE90601C0F6000305F00F054FF0030806
:1029F800D3E90823FEF7D6F9CDE91201BDB147F2B4
:102A08003837DDE90C23C0F6000715F0010F104632
:102A1800194607D0D7E9002308F10108FEF798F80E
:102A280002460B4608376D10EFD1CDE90C23DDE9DE
:102A38000C23DDE91201FEF7B5F9CDE90C0118996F
:102A4800002900F0DE8040F20003DDE90C010022DD
:102A5800C3F6F0734FF0000502F070FD08B14FF0B7
:102A68000105089A002AD4BF002505F00105002DAC
:102A780000F0C780119B002B40F3F58040F2000363
:102A88000022C4F22403DDE90C01FEF761F8CDE968
:102A98000C0108F10100711E1291FDF7F3FF0246C7
:102AA8000B46DDE90C01FEF753F840F20003002263
:102AB800C4F21C03FDF79AFEDDF844C08046A1F17C
:102AC8005079169B002B00F0AD8347F2602340F24B
:102AD8000001C0F60003002003EBCC03C3F6E0714D
:102AE800CDF80CC053E90223FEF75CF942464B4689
:102AF800109DFDF779FE80468946DDE90C01FEF759
:102B080039FA0746FDF7BEFF02460B46DDE90C0120
:102B1800FDF76AFE07F13003CDE90C01404605F8E0
:102B2800013B4946DDE90C2302F026FD002840F070
:102B3800138240F20001DDE90C230020C3F6F07196
:102B4800FDF752FE02460B464046494602F014FD88
:102B5800DDF80CC0002840F0E783BCF1010F40F31A
:102B68008280CDF868B00127CDF870A01D96664622
:102B7800DDE90CAB0C9410E040F200010020C3F634
:102B8800F071FDF731FE42464B4602F0D7FC0028B3
:102B980040F0C783B74280F28B8440F2000340467E
:102BA80049460022C4F224030135FDF7D1FF40F263
:102BB80000030022C4F22403804689465046594641
:102BC800FDF7C6FF8B468246FEF7D4F90446FDF7AB
:102BD80059FF303402460B4650465946FDF704FE6D
:102BE800109A4B46D4554246013782468B4602F02E
:102BF800A5FC52465B460028BED0DDF868B00C9CA8
:102C0800AAE14046FDF73EFFDDE90C23FDF7A0FFF2
:102C180040F200030022C4F21C03FDF7E7FD089A06
:102C2800A1F150758046A946002A40F0EC8240F296
:102C38000003DDE90C010022C4F21403FDF7D4FD02
:102C480042462B46CDE90C0102F096FC002840F0E4
:102C58004A824246DDE90C0105F1004302F06EFCB0
:102C6800002840F0D581DDE906891E9B6FEA03073D
:102C78004FEAD7770E2ECCBF002707F00107002FA9
:102C880000F0B7802B9847F26023C0F6000308993C
:102C980003EBC603C20F0029CCBF002202F00102D9
:102CA800D3E90001CDE90401002A40F0A0810246E1
:102CB8000B4640464946FEF775F8109DFEF75AF94F
:102CC8008246FDF7DFFEDDE90423FDF741FF0246FA
:102CD8000B4640464946FDF787FD0AF1300305F8E3
:102CE800013B089A012A8046894652D040F20003E7
:102CF8000022C4F22403FDF72BFF00220023CDE9B4
:102D0800060102F011FC002840F0EB8110984FF00A
:102D18000108CDF82CB0A346871C0F96DDF820904B
:102D2800DDE906450AE0FDF713FF0022002304460B
:102D38000D4602F0F9FB002840F0CE81DDE90423BE
:102D48002046294608F10108FEF72CF83E46FEF712
:102D580011F98246FDF796FEDDE90423FDF7F8FE3A
:102D680002460B4620462946FDF73EFD00220AF1A1
:102D7800300C07F801CC0137C14540F20003C4F21A
:102D88002403D0D135465C460F9E8046DDF82CB032
:102D9800894642464B4640464946FDF727FD804650
:102DA80089464246DDE904014B4602F0C7FB60B99B
:102DB800DDE9040142464B4602F0B6FB002800F06C
:102DC80090811AF0010F00F08C81109900E01D46E7
:102DD80015F8012C6B1E392A40F067838B42F6D117
:102DE80010993023013631220B70109B1A701296FD
:102DF800B2E0169A002A40F0DF80159F0F9D0C92D2
:102E0800002DD4BF00230123BAF1000FD4BF002343
:102E180003F001034BB1AA45B4BF53462B460F98A4
:102E2800C3EB0A0AED1AC01A0F90159900291CDD88
:102E3800169A002A00F0E982002F12DD0C993A4612
:102E4800204601F073FD5A460C9020460C9901F07B
:102E580085FC594603462046039301F0EBFA039B91
:102E68009B46159BDA1B40F011830121204601F097
:102E78000FFD06901798002805DD06992046179A39
:102E880001F054FD06902A99012940F30A81002790
:102E9800179B002B40F061820123534413F01F035A
:102EA80040F02A811C230F9A9A44ED18D2180F92E9
:102EB8000F9B002B05DD59461A46204601F0F0FB12
:102EC8008346BAF1000F05DD06995246204601F007
:102ED800E7FB06901898002840F029822A9808995C
:102EE8000228D4BF002301230029CCBF002303F00C
:102EF8000103002B00F00C81002940F08C80052292
:102F08000699089B204601F0CDFC06905846069984
:102F180001F056F900287EDD109D01360027DDF806
:102F280030A0312305F8013B0699204601F082FACA
:102F3800BAF1000F00F0D5803B1E18BF012357459A
:102F48000CBF002303F00103002B40F0D080514652
:102F5800204601F06FFA12962046594601F06AFAA7
:102F6800129A531C00222A702C982E99036000296B
:102F780000F0D4812E9A1098156012E4102000F009
:102F880091FCC66046608660066006466062FFF790
:102F9800D2BB0F98714200221591801B17920F9097
:102FA8008AE40021013E189172E4DDE906234FF01E
:102FB8000208CDE9122321E52A98012840F36C8202
:102FC800089A1598531E9842C0F25882C71A089B4F
:102FD800002BA8BF0F9DC0F273820F9A20460121D3
:102FE8009A44D2180F9201F053FC0C9008E7089B02
:102FF80073B940F200030022C4F21403DDE90401AE
:10300800FDF7A6FD42464B4602F0ACFA00286AD00E
:10301800002206920C922B9B0027DDF830A0DE439D
:10302800109D81E7002116912B98002840F39F817D
:103038002B98014611900890656A002217296A604A
:1030480040F2AB8204235B00013203F11400884292
:10305800F9D9089B6A600E2B8CBF002707F001077F
:103068009DE4012216922B9BF3181193591C0029F9
:10307800C8BF0891E0DC0E298CBF002707F00107C4
:10308800089189E401231693CEE700221692EAE715
:103098004FF0FF33002701201193169008932B97C8
:1030A8007AE4B8F1000F7FF4F2AE29F07F4323F4FD
:1030B8007003002B7FF4EBAE40F20003C7F6F07309
:1030C80009EA0303002B3FF4E2AE0F9A0AF1010A62
:1030D800012701320F92DBE635465C460F9EDDF88C
:1030E8002CB0129638E7002006900C9014E7394669
:1030F800204601F09FF92AE7C3F12003042B40F38F
:1031080054820F99043B9A44ED18C9180F91CFE6E1
:103118001699002900F03181002D05DD0C992A4609
:10312800204601F0BDFA0C90002F40F0EA81DDF84E
:1031380030A0109D012308F001000C9F11900F95FD
:103148001D460C9606995846FFF75AFA394630300C
:103158000B90584601F034F8069952460646204628
:1031680001F022FAC3688046002B3DD04FF00109D8
:103178004146204601F05EF92A9959EA010103D136
:10318800119A002A00F0EB81002EC0F29E812A9A43
:10319800324303D1119B002B00F09781B9F1000F46
:1031A80000F3CE810F990B9A01F8012B089B0F9120
:1031B8009D4200F0C28159460A220023204601F0B0
:1031C80071FB57453946834614D00A22002320460E
:1031D800013501F067FB51460A22002307462046C5
:1031E80001F060FB8246ADE75846414600F0E8FF33
:1031F8008146BDE720460A220023013501F052FB33
:10320800074682469EE71296DDF820C059E47542CB
:10321800002D40F00181DDE906014FF00208CDE9FB
:103228000C010CE447F260214246C0F600014B460F
:1032380001EBCC01CDF80CC0109D51E90201FDF75E
:1032480087FCCDE91A01DDE90C01FDF793FE07467D
:10325800FDF718FC0B460246DDE90C01FDF7C4FA40
:1032680007F13003CDE90C0105F8013BDDF80CC08E
:10327800BCF1010F29D0D146DDE90C01B246109E00
:103288001C9501276546A04640F200030022C4F2BF
:103298002403FDF75DFCCDE90C01FDF76BFE044648
:1032A800FDF7F0FB303402460B46DDE90C01FDF773
:1032B8009BFAF4550137AF42E6D11C9D013F5646B3
:1032C8004446CA46ED19CDE90C0140F2000300223C
:1032D800C3F6E073DDE91A01FDF788FA02460B46EA
:1032E800DDE90C0102F048F9F0B940F20001DDE92E
:1032F8001A230020C3F6E071FDF776FA02460B4662
:10330800DDE90C0102F01AF900283FF4ACAC2B46B9
:103318001D4613F8012D302AFAD01DE61098FFF744
:1033280040BADDF868B00C9C129E109950E55846DA
:10333800069900F045FF0028BFF6D0AD5946204653
:103348000A22002301F0AEFA1699013E83460029AD
:1033580040F01981119A0892C0E50698036900EBBC
:103368008303186900F0DAFEC0F1200395E5012116
:10337800119108912B91FFF70FBB109DB146169F35
:10338800AA46DDF81880089E02E001F08BFA834611
:1033980041465846FFF734F901350A2200235946B9
:1033A80000F1300C0AF807C001372046BE42ECDCB9
:1033B800DDF830A04E460027CDF82CC05946012232
:1033C800204601F06DF90699834600F0F9FE0028C1
:1033D8000FDD109900E01D4615F8012C6B1E392AE7
:1033E80040F08C808B42F6D11099312301360B7056
:1033F8009AE503D10B9810F0010FEAD12B461D4630
:1034080013F8012D302AFAD08EE55946159A204630
:1034180001F08CFA834628E505F00F0347F2602295
:10342800C0F60002DDE9060102EBC303D3E900237D
:10343800FDF78EFB2D1108BF4FF00208CDE90C01F6
:103448003FF4FDAA47F23837DDE90C234FF00208B4
:10345800C0F6000715F0010F1046194607D0D7E946
:10346800002308F10108FDF773FB02460B460837F5
:103478006D10EFD1CDE90C23FFF7E1BA1599179A32
:103488005B1AC918D21815911792A0E5594620461B
:1034980001F04CFA8346E8E41999002947D003F56E
:1034A8008663159F03330F9D97E50132D2B29DE4E1
:1034B800DDF868B0DDF870A01D9E0C9CFFF7D3BB4B
:1034C8000F99002308980D1A87E5B9F1000F0F9D91
:1034D8000C9E0FDD59460122204601F0E1F80699BD
:1034E800834600F06DFE002847DD0B99392931D05D
:1034F80001310B910B9A05F8012B15E501321A7071
:1035080012E50C9A2046516800F0B0FF0C9B03F1BD
:103518000C011A690232920005460C3000F0D6FC04
:1035280020462946012201F0BBF8824601E61F9B8E
:10353800159F0F9DC3F136034FE50F9D0C9E3DE788
:103548000B9B0F9D392B0C9E04D00B98431C05F840
:10355800013BE9E4392305F8013B10993CE70B9856
:1035680033460F9D39280C9EF4D0002B01DD013025
:103578000B900B9905F8011BD6E4BBD10B9810F002
:10358800010FB7D0B1E700230C9920460A2201F0B9
:1035980089F9119B08930C90A0E408990E298CBF17
:1035A800002707F00107FFF7FAB93FF481AC1C3395
:1035B80079E40127FFF78AB9F8B540F2F404C2F2BA
:1035C80000040F46054600F0A5FDA3685E6826F0D6
:1035D800030606F57E630F33DF1B3F0B013F3F03F6
:1035E800B7F5805F07DB0021284601F03DFCA368A2
:1035F800F318834204D0284600F08EFD0020F8BD61
:103608007942284601F030FCB0F1FF3F10D0A268A3
:1036180040F21053C2F20003F61B46F0010628469A
:1036280056601A68D71B1F6000F076FD0120F8BDB0
:103638000021284601F018FCA368C21A0F2ADADD17
:1036480040F2FC4440F21051C2F20004C2F2000100
:1036580042F001022468001B08605A60CBE700BFF3
:103668002DE9F04105460C46002900F0888000F05D
:1036780051FDA4F1080240F2F4005668C2F20000BD
:1036880026F00103D0F808C0D1188C454F6827F000
:10369800030700F0958016F001064F605FD0002602
:1036A800CC19646814F0010F06D1DB19002E7AD00A
:1036B8008C68C9688C60E16043F00101D3505160A7
:1036C800002E47D1B3F5007F5BD3590A04299EBF6A
:1036D8004FEA931C0CF1380C4FEACC0428D9142972
:1036E8009CBF01F15B0C4FEACC0421D954299EBF41
:1036F8004FEA133C0CF16E0C4FEACC0418D9B1F523
:10370800AA7F9EBF4FEAD33C0CF1770C4FEACC045A
:103718000ED940F2545C614595BF4FEA934C4FF483
:103728007C740CF17C0C4FF07E0C98BF4FEACC04F3
:103738000419A168A14203D164E089688C4204D0CD
:10374800486820F003008342F7D3CB68D3609160C8
:10375800CA609A602846BDE8F04100F0DDBC54F824
:10376800084C00F1080C121B1B199468644547D0DB
:10377800D2F80CC0CCF80840C4F80CC090E7BDE8FB
:10378800F081DB084FF0010C466800EBC3019B1089
:103798000CFA03F3D1608C6846EA03034360946033
:1037A800E2608A60D6E78C681C4FBC4281D1D35056
:1037B80043F00103E260A26053609460D460C9E7FB
:1037C800FB1816F0010F07D154F8081C521A5B18A1
:1037D800D4689168A160CC6040F200518260C2F266
:1037E800000143F0010050600A689342B2D340F2EE
:1037F8000C532846C2F200031968FFF7DDFEA9E75B
:1038080001264DE7012644684FEAAC0C0B4606FA40
:103818000CFC44EA0C04446098E700BFFC0000205C
:1038280047F22823C0F6000318687047004870471D
:103838002C720008004870472C72000870B50546C5
:103848000E46144672B147F2E0511046C0F6000128
:1038580001F01EFB58B947F2E0502C62C0F6000098
:10386800EE6170BD47F2E050C0F6000070BD47F24F
:103878009C512046C0F6000101F00AFB0028EAD05E
:10388800002070BD40F200030A46C2F20003014660
:103898001868D3E740F200030146C2F20003186833
:1038A800FFF7DEBE40F200030146C2F200031868CB
:1038B80000F000B82DE9F04F01F10B04162C83B08D
:1038C80006462FD8002310248C422CBF194643F0FB
:1038D8000101002930D1304600F01CFCB4F5FC7F12
:1038E8002ED24FEAD40E40F2F405C2F2000505EBE1
:1038F800CE02D368934200F006825A6803F10805A5
:10390800D968304622F0030C9A6863445C688A6080
:1039180044F00104D1605C6000F0FEFB284603B06F
:10392800BDE8F08F24F00704E30F8C422CBF194642
:1039380043F001010029CED00C2300253360EDE7C8
:103948005FEA542E04BF4FEAD40E4FEACE0040F08F
:10395800908040F2F405C2F200052818C368984226
:1039680006D10DE0002A80F26F81DB68984207D00B
:10397800596821F003010A1B0F2AF3DD0EF1FF3EFF
:103988000EF1010E40F2F407C2F2000707F1080138
:103998008B68994208BF7A6826D05A6822F0030CCF
:1039A800C4EB0C020F2A00F39481002AC9608960D5
:1039B80080F29980BCF5007F80F065814FEADC0CCD
:1039C8004FF0010A7A6807EBCC004FEAAC0C0AFA10
:1039D8000CFCD860D0F808804CEA02027A60C3F880
:1039E8000880C8F80C3083604FF0010C4FEAAE0332
:1039F8000CFA03FC944500F2828012EA0C0F08D1FD
:103A08002EF0030E4FEA4C0C0EF1040E12EA0C0FC6
:103A1800F8D007EBCE09F246C846D8F80C309845DE
:103A280007D168E1002A80F27881DB68984500F0C8
:103A38006281586820F00300021B0F2AF2DD1D4640
:103A48001F19D3F80CC044F0010E55F8084F304642
:103A5800BA5042F00102C3F804E0CCF80840C4F8B8
:103A68000CC08F60CF607A60B960F96000F054FBD9
:103A780054E7BEF1040F9EBF4FEA941E0EF1380EB4
:103A88004FEACE007FF665AFBEF1140F9CBF0EF172
:103A98005B0E4FEACE007FF65CAFBEF1540F9EBFBF
:103AA8004FEA143E0EF16E0E4FEACE007FF651AF8C
:103AB800BEF5AA7F9EBF4FEAD43E0EF1770E4FEABD
:103AC800CE007FF646AF40F254539E4595BF4FEA6D
:103AD800944E4FF47C700EF17C0E4FF07E0E98BF22
:103AE8004FEACE0035E703EB0C0203F10805304638
:103AF800536843F00103536000F00EFB0EE7D7F85C
:103B08000880D8F8043023F00309C4EB09024C45B7
:103B180094BF002301230F2AD8BF43F00103002BD1
:103B280000F0A18040F20C5BD5F80824C2F2000B2B
:103B3800DBF8003010331B19B2F1FF3F06D003F554
:103B48007E631F3323F47E6323F01F031946304638
:103B5800019301F089F9019BB0F1FF3F824600F023
:103B6800F48008EB0901814200F2EC80DBF80420C4
:103B78009A185145CBF8042000F04581D5F808542F
:103B880040F2F400C2F20000B5F1FF3F08BFC0F8F0
:103B980008A403D05244511ACBF804101AF00705B0
:103BA800304617BFC5F108054FF48055AA4405F5FE
:103BB800805553441B051B0DED1A294601F054F995
:103BC800B0F1FF3F00F02C81CAEB0001491941F028
:103BD8000101DBF8042040F20C53C7F808A0C2F238
:103BE8000003AA18B845CBF80420CAF8041017D067
:103BF800B9F10F0F40F2DF80A9F10C01052521F082
:103C0800070108EB01000F2985604560D8F804001A
:103C180000F0010041EA0000C8F8040000F2AC809E
:103C2800D04640F20C53DBF82C10C2F200038A4253
:103C3800DBF8301088BFDA6240F20C53C2F200039E
:103C48008A4288BF1A6382E05C189A68D96830464D
:103C5800666803F108058A6046F00103D160636075
:103C680000F05AFA5AE608EB040342F0010244F065
:103C780001043046C8F8044008F108055A60BB60E2
:103C880000F04AFA4AE64FEA5C22042A54D9142A78
:103C980000F289805B324FEAC208A84440F2F40778
:103CA800C2F20007D8F80800404503D16FE08068E9
:103CB800804504D0426822F003029445F7D3D0F837
:103CC8000CC0C3F80CC098607A68C360CCF80830A0
:103CD8008AE61F19304644F00104CF605C6003F1A6
:103CE8000805BA5042F001028F607A60B960F96045
:103CF80000F012FA12E60AF1010A1AF0030F5FD077
:103D080003F1080889E603F10802D3689A4208BF5C
:103D18000EF1020E3FF436AEEFE51D461918DA68CB
:103D2800304655F8083F4C68936044F00104DA6067
:103D38004C6000F0F1F9F1E54FEA9C1238324FEA95
:103D4800C208AAE7B8453FF411AFD7F80880D8F8F9
:103D5800042022F00302944294BF00230123121B83
:103D68000F2AD8BF43F00103002B3FF47CAF304645
:103D7800002500F0D1F9D1E508F10801304601939A
:103D8800FFF76EFC019BD7F808805A6849E74FF0A7
:103D9800010AD7F80480921084460AFA02F248EA27
:103DA80002027A608DE7542A24D84FEA1C326E3218
:103DB8004FEAC20871E70123D046CAF80430C6E7C3
:103DC8004A461EF0030F13460EF1FF3E33D053F858
:103DD80008299A42F5D07B684FEA4C0C9C453FF67F
:103DE8008EAEBCF1000F3FF48AAE1CEA030F27D059
:103DF800D6460EE6B2F5AA7F15D84FEADC327732FE
:103E08004FEAC20849E70805000D00287FF4B6AE5E
:103E1800D7F808804B4443F00103C8F8043000E7A2
:103E280001210025D5E640F2545082420DD94FF4C5
:103E38007C787E2231E77B6823EA0C037B60CBE742
:103E48004FEA4C0C0AF1040ACFE74FEA9C427C3255
:103E58004FEAC20821E700BF10F0030FC9B210B43F
:103E680010D0002A2FD003788B422AD0013A05E0DF
:103E7800002A28D00378013A8B4222D0013010F072
:103E8800030FF5D1032A11D941EA012444EA044475
:103E9800036884EA0303A3F1013C2CEA030313F04B
:103EA800803F03D1043A0430032AF1D85AB1037889
:103EB8008B4206D0013A32B110F8013F013A8B42E9
:103EC800F9D110BC70470020FBE700BF032A2DE999
:103ED800F0070BD83AB1002311F803C000F803C06B
:103EE80001339342F8D1BDE8F007704782180C46B9
:103EF800034603E014F8011C03F8011C03F0030651
:103F08001946A44601330134002EF3D11CF00304F2
:103F1800634608BFC1EB020C68D06542C4F1040ACD
:103F28000CEB050733464FEACA0A5CF805604FEA0E
:103F3800C408551A08E057F8044F264604FA0AF44C
:103F480049EA0404CC5004335C18032D26FA08F916
:103F5800A5F104050CEB0306EDDC002302E0F15C9F
:103F6800E154013319199142F9D3BCE753F8404C95
:103F780041F8404C53F83C4C41F83C4C53F8384C11
:103F880041F8384C53F8344C41F8344C53F8304C21
:103F980041F8304C53F82C4C41F82C4C53F8284C31
:103FA80041F8284C53F8244C41F8244C53F8204C41
:103FB80041F8204C53F81C4C41F81C4C53F8184C51
:103FC80041F8184C53F8144C41F8144C53F8104C61
:103FD80041F8104C53F80C4C41F80C4C53F8084C71
:103FE80041F8084C53F8044C41F8044C1C460D4663
:103FF80040334031BCF13F0FACF1400CB6DC2146F8
:104008002B46541B0FE051F8105C43F8105C51F834
:104018000C5C43F80C5C51F8085C43F8085C51F8F8
:10402800045C43F8045C0F2C0D469C4601F110011A
:1040380003F11003A4F11004E5DCCCEB020100232A
:1040480003E0EC584CF8034004335E19032903EBF2
:104058000C04A1F10401F4DC7FE700BF88428C4620
:1040680070B4054614460ED98B1898420BD242B14B
:10407800C2EB030C0146531E1CF80320CA54013B33
:10408800FAD270BC70470F2A09D8002CF9D0002347
:104098001CF80320EA540133A342F9D1F1E741EABD
:1040A800000313F0030FF0D194460C46034625682D
:1040B800ACF1100C1D6065685D60A5689D60E568E1
:1040C8001034DD601033BCF10F0FF0D8103A4FEA0E
:1040D800121C0CF10105CCEB0C7C2D0102EB0C162B
:1040E80001EB050C4519032E3446CED900235CF8A4
:1040F8000320EA500433F21A032AF8D8043EB3081E
:104108005A1CC3EB83739200944406EB8304AD18E6
:10411800BBE700BF704700BF704700BF020C0346F3
:104128001204B2B1002013F07F4F01D108301B02F6
:1041380013F0704F01D104301B0113F0404F01D12F
:1041480002309B00002B03DB13F0804F04D00130BA
:10415800704703041020E6E72020704703680246F2
:1041680013F0070009D013F0010F21D113F0020F4B
:1041780022D19B0802201360704799B209B91B0C21
:10418800102013F0FF0F01D108301B0A13F00F0F96
:1041980001D104301B0913F0030F01D102309B0831
:1041A80013F0010F02D15B0804D00130136070478F
:1041B80000207047202070475B080120136070477B
:1041C80003460A69006910B4801A11D1043203F158
:1041D800140C92009B1889180431043353F8044CCA
:1041E800043B51F8042C0439944203D19C45F5D37F
:1041F80010BC704738BF4FF0FF30F9D30120F7E704
:1042080040F20003C7F6F07301EA0303A3F1507309
:10421800002B02DD1946002070475B421B15132B4B
:104228000EDD143B1E2B03DD0123002118467047C9
:104238000122C3F11F03002112FA03F31846704745
:104248004FF40022002052FA03F170472DE9F041A3
:10425800046900F114060F46043450F8245000EBAA
:104268008404A0462846FFF759FF0A28C0F1200316
:104278003B6014DCA642C0F10B0337D254F8041C8F
:10428800D94025FA03FC15304CF07E53854043F4A1
:10429800E00341EA050210461946BDE8F081A6424E
:1042A80020D300210B3802BF45F07E530A4643F461
:1042B800E003F0D0B442C0F1200319D954F8044CFB
:1042C800DC40854021FA03FC45F07E5511FA00F0E8
:1042D80045F4E00544EA000245EA0C031046194695
:1042E800BDE8F08154F8041C043CDBE70021C8E772
:1042F8000024E6E72DE9F04383B00E4601A90746FE
:10430800FFF7A4FF0D46044669463046FFF79EFFB7
:10431800DDF804C0A946A0460B4602463169164698
:1043280038691F46401A0099C1EB0C0101EB401196
:104338000029C9BF05EB0159A3EB015724464D4697
:10434800DCBF12463B4620462946FCF72BFD03B04E
:10435800BDE8F083172810B504460EDD40F20001D1
:104368000020C3F6F07140F200030022C4F22403D7
:10437800FCF7EEFB013CF6D110BD47F26023C0F616
:10438800000303EBC003D3E9000110BD1369013931
:1043980002F1140C10B402EB83024C1114320134F4
:1043A800944500EB84040FD200235CF80310C1503D
:1043B800043303EB0C018A42F7D86FEA0C0C624411
:1043C80022F0030204328018844204D9002340F802
:1043D800043B8442FBD810BC704700BF02694B11F4
:1043E8009A4210DB0EDD11F01F010BD01A4600EBCC
:1043F80083035B6923FA01FC0CFA01F1994202D0AC
:10440800012070471A46043200F1140100EB8203C0
:1044180003F1040C61450BD250F82220002AEFD199
:10442800994205D253F8042D002AE9D19942F9D3CB
:104438000020704730B5456A83B0044655B139B19C
:10444800636A4A68DB6853F82200086043F8221060
:1044580003B030BD10200191FFF724FA0199606282
:10446800C560456085600560E9E700BF70B5446ACE
:1044780006460D4664B1E268A2B152F82530EBB1A8
:10448800196842F825100022DA601A61184670BDD2
:104498001020FFF707FA002304467062C3604360E8
:1044A8008360036010223046042100F00FFE736A17
:1044B800E060DA68002AE0D11346E7E701243046D5
:1044C8002146AC40621D920000F000FE0346002821
:1044D800DCD045608460D6E72DE9F04583B0012142
:1044E8001D4614460A9F0B9EFFF7C0FF25F00042A9
:1044F80025F07F4323F4700315465FEA125A0093B0
:104508001CBF43F4801300938046002C23D002A8DC
:1045180040F8044DFFF722FE0346002837D10199E1
:10452800009AC8F81410002A14BF02240124C8F8FD
:104538001820C8F81040BAF1000F1BD0AAF5866AF7
:10454800C3F13502AAF1030A53443B603260404686
:1045580003B0BDE8F0856846FFF700FE01231C465E
:10456800C8F81030009BC8F8143000F12003BAF1E5
:10457800000FE3D108EB8402A3F58663023B3B609E
:104588001069FFF7CBFDC0EB44103060DFE7009AFD
:10459800C0F1200112FA01F1C24001980143C8F8A4
:1045A80014100092BFE700BF2DE9F84F13690F6997
:1045B8000C461546FF1A002F4FD06ADB002701F181
:1045C80014066168FFF752FFD5F81080D4F810C0C0
:1045D80005F11401002205EB880504EB8C0405F1B4
:1045E8001408143400F11403C76051F8047B56F81A
:1045F800045BBB461FFA87FA3F0C1FFA85F9C7EB25
:104608001547CAEB090A524407EB224792B242EA1D
:10461800074243F8042B3A148845E6D8A6420ED23E
:1046280056F8041B8DB2090C521901EB224192B2C3
:1046380042EA014243F8042B0A14B442F0D853F872
:10464800042C32B953F8082C0CF1FF3C043B002A27
:10465800F8D0C0F810C0BDE8F88F043301F1140693
:104668009B00D218CB180433043253F804CC043B13
:1046780052F8041C043A8C450AD19E42F5D3002115
:10468800FFF7F4FE0123036100234361BDE8F88FBF
:1046980097D223462C4601271D4604F1140690E7BD
:1046A8002DE9F8450D698B68561101350C46AD1991
:1046B80090469D428246496803DD5B0001319D4278
:1046C800FBDC5046FFF7D2FE002E074600F114022D
:1046D8000ADD0023194642F823100133B342FAD108
:1046E80007EB830303F11402206904F1140304EBBC
:1046F8008000143018F01F081BD0C8F1200E0021CC
:104708001E6806FA08FC41EA0C0142F8041B53F83B
:10471800041B984221FA0EF1F2D8116001B101355B
:104728005046013D21463D61FFF784FE3846BDE80D
:10473800F88553F8081042F8081008F1040808EB47
:1047480003018842ECD953F8081042F8081008F120
:10475800040808EB03018842EBD8E1E72DE9F04FA4
:10476800D1F8108017690D46164687B0B845B5BF11
:1047780015463B460B464746B4BF1E469846AB68AF
:1047880008EB070469689C42C8BF0131FFF76EFE59
:1047980000EB840300F1140B143303909B4504933E
:1047A80006D204995B46002243F8042B9942FBD8B1
:1047B80006EB880806F1140908F1140805EB870CC4
:1047C8001435C145CDF804800CF1140C02954BD278
:1047D8004FF0000A059459F80A400AEB0B08A0B2FA
:1047E800D8B1029A4346002452F8045B1968AFB264
:1047F8002D0C8EB2090C00FB076600FB051136195B
:1048080001EB1641B6B20C0C944546EA014643F852
:10481800046BE9D81C6059F80A40240C1CD05BF8DA
:104828000A204146029B002510461E8897B206FBC7
:10483800045505EB104547EA05470F6051F8040F8A
:1048480053F8042B86B2120C02FB046202EB1542E9
:10485800150C9C45E9D80A600AF1040A019A0AEB8A
:1048680009039A42B7D8059C002C0BDD049A52F82C
:10487800043C3BB9134603E053F8082C043B0AB93F
:10488800013CF9D1039B18461C6107B0BDE8F08FC5
:1048980010B50C460121FFF7E9FD012244610261D0
:1048A80010BD00BF2DE9F0450D46002106462C69D4
:1048B80083B005F11408084658F8017001301FFA52
:1048C80087FA4FEA174C0AFB02330CFB02FC0CEB8D
:1048D800134C9BB203EB0C4348F80130043184427B
:1048E8004FEA1C43E8DC3BB1AA68944208DA05EBBE
:1048F800840201342C615361284603B0BDE8F08579
:104908006968304601930131FFF7B0FD2A6905F166
:104918000C010232920007460C30FFF7D7FA2946FD
:1049280030463D46FFF786FD019BE0E72DE9F04163
:10493800154612F00302044688462CD1AD101ED04D
:10494800666A002E34D0B768002F3BD015F0010FEF
:1049580008D16D1013D03E68A6B13046074615F051
:10496800010FF6D041463A462046FFF7F7FE41468A
:1049780006462046FFF75EFD6D10B046EBD1404677
:10498800BDE8F08139463A462046FFF7E7FE386031
:1049980007460660E3E747F2602C0023C0F6000CE8
:1049A8000CEB8202D2F8C420FFF77CFF8046C5E7F3
:1049B8001020FEF777FF002306466062C36043605D
:1049C80083600360204640F27121FFF761FF0023F6
:1049D800B06007460360B9E72DE9F8451E4648F67A
:1049E800396306F1080CC3F6E30388460546174603
:1049F80083FB0C134FEAEC7CCCEB630CBCF1010F8E
:104A080035DD00210122520001319445FBDC2846A6
:104A1800FFF72CFD089B43610123092F036122DD69
:104A280008F1090A092418F8043001460A22013459
:104A3800303B2846FFF736FFA742F4DC0AEB0708AD
:104A4800A8F10808BE420CDD002418F8043001461D
:104A580001340A22303B2846FFF724FFE3199E421F
:104A6800F3DCBDE8F88508F10A080927EAE7002120
:104A7800CDE700BF2DE9F04F914683B007460E46BB
:104A8800002900F03A81A1F1080809F10B04FFF7A9
:104A980041FB162CD8F804100B4600F2A080102217
:104AA800002514464C4538BF45F00105002D40F05F
:104AB8002A8121F0030A9245A2BF4046554608F1D3
:104AC800080875DA40F2F40308EB0A00C2F20003A2
:104AD800D3F808E0864500F01A81D0F804C02CF01D
:104AE800010B8344DBF804B01BF0010F7CD0AC460B
:104AF800284611F0010F40F09B8056F8081CC1EBC6
:104B0800080BDBF8045025F00305002800F0DD80D1
:104B1800704500F01F8105EB0A030CEB0305954275
:104B2800B8BF1D46C0F2D28081685B46C068AAF152
:104B38000402242A8160C86053F8081FDBF80C00BF
:104B48008160C86000F2D080132A9C4621D9314682
:104B58000BF1100C51F8040BCBF8080070680E1D0F
:104B68001B2ACBF80C0014D94868311D0BF1180C1E
:104B7800CBF8100070680E1D242ACBF8140008D159
:104B88004A680BF1200CCBF8182072680836CBF86D
:104B98001C20314698466246584651F8043B42F874
:104BA800043B7368CCF804304B685360DBF804307E
:104BB800C4EB050CBCF10F0F26D8421903F0010312
:104BC80043EA05054560536843F0010353603846DE
:104BD8004546FFF7A1FA284603B0BDE8F08F24F058
:104BE80007042246E50F5DE72CF0030C0CEB0A05E1
:104BF8009542FFF67EAF82680B46C168404608F1D1
:104C080008088A60D160D3E7011903F0010301EBBA
:104C18000C0243EA04044CF0010344604B6038463C
:104C28005368083143F001035360FEF719FDCEE7DE
:104C380049463846FEF73EFE0546002841D0D8F8DA
:104C48000430A0F1080223F0010141448A4200F037
:104C5800D780AAF104023146242A78D8132A0346B9
:104C680021D9344654F8043B211D40F8043B031D68
:104C7800D6F804C01B2AC5F804C014D9D4F804E037
:104C88001C1D01F1040CC0F804E048680CF1040193
:104C98005860231D242A06D1DCF8042062604A6883
:104CA80008315A60083308461A4650F8044B42F84F
:104CB800044B496859604368536031463846FEF7EB
:104CC800CFFC3846FFF728FA85E755449542AFDB15
:104CD8005B46DBF80C00AAF1040253F8081F242AEB
:104CE8008160C8607FF630AF184631469846FFF7B6
:104CF800B5F95846DBF804305AE7114603B0BDE869
:104D0800F04FFEF7D7BD0C2300253B6063E7DEF8C4
:104D1800045004F1100B25F0030C0CEB0A00584565
:104D2800B8BF7046FFF6E5AE08EB0402011B41F080
:104D380001019A6051603846D8F80410354601F0F0
:104D480001031C43C8F80440FFF7E6F943E7FFF7FF
:104D580085F9B2E7554404F11001AC448C45B5DB44
:104D68005D46DBF80C00AAF1040255F8081F242A56
:104D78008160C8604CD8132A284624D931460BF1E3
:104D8800100051F804EBCBF808E0D6F804E00E1D4B
:104D98001B2ACBF80CE016D9D1F804E0311D0BF131
:104DA8001800CBF810E0D6F804E00E1D242ACBF842
:104DB80014E008D14A680BF12000CBF8182072687B
:104DC8000836CBF81C203146024651F804EB42F86D
:104DD80004EB76684660496851600BEB0402C4EB4B
:104DE8000C0141F001019A6051603846DBF804106B
:104DF80001F001031C43CBF80440FFF78DF9EAE604
:104E08005568404608F1080825F003055544CFE6E3
:104E1800314628460093CDF804C0FFF71FF9DDF8A6
:104E280004C0009BD9E700BF0246404240EA0203A3
:104E380021F0004141EAD373C3F1FE4303F5700347
:104E4800584240EA0303D8170130704702464042EF
:104E5800104321F0004141EAD070C0F1FE4000F556
:104E68007000C00F704700BF38B540F24054C2F21E
:104E780000040546084600232360FBF7A1FCB0F1B7
:104E8800FF3F00D038BD2368002BFBD02B6038BD16
:104E980080EA010212F0030F3AD110F0030220F069
:104EA800030021F0030150F804CB08BF51F8043B7C
:104EB8000DD082F003024FEAC2026FF07F4323FA5B
:104EC80002F251F8043B4CEA020C43EA020300BF29
:104ED800ACF101329C4501BF22EA0C0212F0803F7E
:104EE80050F804CB51F8043BF2D04FEA0C604FEA7B
:104EF8001C2C012828BFB0EB036F08BF1B0AF4D095
:104F080003F0FF034FEA1060A0EB0300704700BFF7
:104F180010F0030F0AD010F8012B11F8013B012AF9
:104F280028BF9A42F4D0A2EB030070474DF8045D05
:104F38004DF8044D4FF0010242EA022242EA0242D1
:104F480001F0030C21F0030150F8044B51F8045B05
:104F5800BCF1020F26D04BD824F07F4CBCEB152FA8
:104F6800A4EB020323EA04030DD113EAC21308BF1A
:104F780051F8045B0AD18CEA040CBCEB056F0CD128
:104F880050F8044BE8E74FEA15255CE033F07F431F
:104F980052D10D784FEA146C55E04FEA146C05F0C5
:104FA800FF0550E04FEA044CA4EB02034FEA1C4C07
:104FB80023EA0403BCEB154F17D113EAC21308BF49
:104FC80051F8045B07D18CEA040CBCEB054F08D1FF
:104FD80050F8044BE6E71B042ED10D884FEA144C19
:104FE80031E04FEA05454FEA144C4FEA15452AE0EF
:104FF80004F0FF0CBCEB156FA4EB020323EA0403D7
:105008000DD113EAC21308BF51F8045B0AD18CEA28
:10501800040CBCEB052F0AD150F8044BE8E74FEA23
:10502800156510E014F0FF0F06D051F8045B4FEA45
:10503800142C25F07F4506E04FF000005DF8044B86
:105048005DF8045B70470CF0FF0205F0FF000128D3
:1050580028BF904204BF4FEA1C2C2D0AF3D0A2EBC4
:1050680000005DF8044B5DF8045B704720F0030115
:1050780010F00300C0F1000051F8043B00F1040CEB
:105088004FEACC0C6FF000021CBF22FA0CF213435B
:105098004FF0010C4CEA0C2C4CEA0C4CA3EB0C0224
:1050A80022EA030212EACC1204BF51F8043B04308E
:1050B800F4D013F0FF0F1FBF013013F47F4F0130FE
:1050C80013F47F0F18BF0130704700BF38B501FBDC
:1050D80002F1FEF7EFFB0446F8B150F8042C22F079
:1050E8000302043A242A1AD8132A03460FD90021A6
:1050F80040F8041B031D1B2A616008D91D1D41606F
:1051080059602B1D242A02BF6960596008331A466A
:10511800002142F8041B59605160204638BD002127
:1051280000F002F8204638BD032AC9B230B407D8C7
:1051380022B10023C15401339342FBD130BC7047E4
:1051480000EB020C034601E003F8011C03F0030422
:105158001A460133002CF7D14FF00133C2EB0C048F
:1051680003FB01F31FE042F8403C42F83C3C42F8A4
:10517800383C42F8343C42F8303C42F82C3C42F887
:10518800283C42F8243C42F8203C42F81C3C42F8B7
:10519800183C42F8143C42F8103C42F80C3C42F8E7
:1051A800083C42F8043C154640323F2CA4F1400428
:1051B800D9DC2A46C5EB0C0407E042F8103C42F85B
:1051C8000C3C42F8083C42F8043C154610320F2CBF
:1051D800A4F11004F1DC2A46C5EB0C0501E042F805
:1051E800043C14460432032DA5F10405F7DC01E064
:1051F80004F8011B6445FBD3A0E700BF00000000D2
:105208004A1E08BF7047C0F02481884240F21681C8
:10521800114200F01781B0FA80F3B1FA81F2A2EBE3
:105228000303C3F11F0304A202EB03134FF00002B0
:105238009F4600BFAFF30080B0EBC17F00BF42EBD9
:10524800020228BFA0EBC170B0EB817F00BF42EB28
:10525800020228BFA0EB8170B0EB417F00BF42EB98
:10526800020228BFA0EB4170B0EB017F00BF42EB08
:10527800020228BFA0EB0170B0EBC16F00BF42EB88
:10528800020228BFA0EBC160B0EB816F00BF42EB08
:10529800020228BFA0EB8160B0EB416F00BF42EB78
:1052A800020228BFA0EB4160B0EB016F00BF42EBE8
:1052B800020228BFA0EB0160B0EBC15F00BF42EB68
:1052C800020228BFA0EBC150B0EB815F00BF42EBE8
:1052D800020228BFA0EB8150B0EB415F00BF42EB58
:1052E800020228BFA0EB4150B0EB015F00BF42EBC8
:1052F800020228BFA0EB0150B0EBC14F00BF42EB48
:10530800020228BFA0EBC140B0EB814F00BF42EBC7
:10531800020228BFA0EB8140B0EB414F00BF42EB37
:10532800020228BFA0EB4140B0EB014F00BF42EBA7
:10533800020228BFA0EB0140B0EBC13F00BF42EB27
:10534800020228BFA0EBC130B0EB813F00BF42EBA7
:10535800020228BFA0EB8130B0EB413F00BF42EB17
:10536800020228BFA0EB4130B0EB013F00BF42EB87
:10537800020228BFA0EB0130B0EBC12F00BF42EB07
:10538800020228BFA0EBC120B0EB812F00BF42EB87
:10539800020228BFA0EB8120B0EB412F00BF42EBF7
:1053A800020228BFA0EB4120B0EB012F00BF42EB67
:1053B800020228BFA0EB0120B0EBC11F00BF42EBE7
:1053C800020228BFA0EBC110B0EB811F00BF42EB67
:1053D800020228BFA0EB8110B0EB411F00BF42EBD7
:1053E800020228BFA0EB4110B0EB011F00BF42EB47
:1053F800020228BFA0EB0110B0EBC10F00BF42EBC7
:10540800020228BFA0EBC100B0EB810F00BF42EB46
:10541800020228BFA0EB8100B0EB410F00BF42EBB6
:10542800020228BFA0EB4100B0EB010F00BF42EB26
:10543800020228BFA0EB0100104670470CBF0120F4
:1054480000207047B1FA81F2C2F11F0220FA02F07F
:10545800704708B14FF0FF3000F00EB80029F8D0BF
:105468002DE90340FFF7CCFEBDE8064002FB00F340
:10547800A1EB0301704700BF704700BF4FF0FF3C2E
:1054880006E000BF4FF0010C02E000BF4FF0010C36
:105498004DF804CD4FEA410C7FEA6C5C4FEA430CAF
:1054A80018BF7FEA6C5C1BD001B050EA410C0CBFFE
:1054B80052EA430C91EA030F02BF90EA020F002060
:1054C800704710F1000F91EA030F58BF994208BFC7
:1054D80090422CBFD8176FEAE37040F00100704784
:1054E8004FEA410C7FEA6C5C02D150EA013C07D1DB
:1054F8004FEA430C7FEA6C5CD6D152EA033CD3D026
:105508005DF8040B704700BF8446104662468C461F
:105518001946634600E000BF01B5FFF7B7FF002852
:1055280048BF10F1000F01BD4DF808EDFFF7F4FF7B
:105538000CBF012000205DF808FB00BF4DF808ED06
:10554800FFF7EAFF34BF012000205DF808FB00BF29
:105558004DF808EDFFF7E0FF94BF012000205DF84B
:1055680008FB00BF4DF808EDFFF7CEFF94BF012000
:1055780000205DF808FB00BF4DF808EDFFF7C4FFF9
:1055880034BF012000205DF808FB00BF4BB942B9C9
:10559800002908BF002802D04FF0FF310846FFF766
:1055A8006BBF82B0EC462DE9005000F005F8DDF83D
:1055B80004E002B00CBC7047F8B514461D46064618
:1055C8000F4600F0D7F900FB05F5A0FB042304FB08
:1055D8000154E318B61A67EB0307069BC3E9006793
:1055E800F8BD00BFF8B514461D4606460F4600F044
:1055F8000FF800FB05F5A0FB042304FB0154E31896
:10560800B61A67EB0307069BC3E90067F8BD00BF3E
:1056180000292DE9F04F85B0C0F2C8800026002B84
:10562800C0F2BF808946144605469B46002B4AD1E6
:105638008A4257D9B2FA82F353B1C3F1200001FA72
:1056480003F925FA00F812FA03F49D4048EA09091B
:10565800270C484639461FFA84FBFFF7D1FD394627
:1056680082464846FFF7FAFE2A0C0BFB0AF342EA89
:1056780001494B4509D919EB04090AF1FF3A04D24B
:105688004B4584BF0AF1FF3AA144C3EB09093946E7
:105698004846ADB2FFF7B4FD394680464846FFF7A5
:1056A800DDFE0BFB08FB45EA0145AB4507D92D1983
:1056B80008F1FF3803D2AB4588BF08F1FF3848EA44
:1056C8000A48002703E08B4257D90027B8464246CC
:1056D8003B4616B1524263EB43031946104605B0E8
:1056E800BDE8F08F22B911460120FFF789FD044675
:1056F800B4FA84F8B8F1000F5ED1C4EB0908270C9E
:105708001FFA84F90121029139464046FFF778FDD6
:10571800394682464046FFF7A1FE4FEA154809FB85
:105728000AF348EA014B5B4509D91BEB040B0AF164
:10573800FF3A04D25B4584BF0AF1FF3AA344C3EBA6
:105748000B0B39465846ADB2FFF75AFD394680462D
:105758005846FFF783FE09FB08F945EA0145A945C4
:1057680007D92D1908F1FF3803D2A94588BF08F1D8
:10577800FF3848EA0A48029FA9E7B3FA83F7002FDF
:1057880068D18B422CBF4FF000094FF001098242CB
:105798008CBF4C4649F00104002C96D04FF001080C
:1057A80095E7524263EB4303F6433BE7404261EB24
:1057B80041014FF0FF3632E704FA08F4C8F1200738
:1057C80035FA07F329FA07FA270C09FA08FB3946CC
:1057D800504643EA0B020292FFF712FD39461FFAC0
:1057E80084F983465046FFF739FE029809FB0BF20D
:1057F800030C43EA01439A4204D91B190BF1FF3BFE
:10580800C0F0B1809B1A394618460193FFF7F8FC9F
:105818000199824608463946FFF720FEDDF808C0A0
:1058280009FB0AF31FFA8CF040EA0142934208D9B7
:1058380012190AF1FF3A04D2934284BF0AF1FF3ADF
:10584800121905FA08F54AEA0B4EC3EB0208CDF81F
:1058580008E059E7C7F1200003FA07FAC24035FA11
:1058680000F342EA0A0B21FA00F801FA07F9404668
:105878004FEA1B4A43EA0901029151461FFA8BF28B
:105888000392FFF7BDFC514681464046FFF7E6FD0F
:10589800039BDDF808C003FB09F24FEA1C4014FA29
:1058A80007F340EA0144A24204D914EB0B0409F1BE
:1058B800FF3952D3A41A514620460193FFF7A0FCA2
:1058C800514680462046FFF7C9FD0398DDF808C019
:1058D80000FB08F21FFA8CF343EA0140019B824265
:1058E80004D910EB0B0008F1FF3830D348EA094817
:1058F8001FFA83FC1B0C801A1FFA88FE4FEA184A0D
:105908000CFB0EF90CFB0AFC03FB0EC103FB0AF2AD
:1059180001EB19418C4588BF02F5803202EB114E2C
:10592800704510D31FFA89F905FA07F709EB01400A
:1059380014BF0022012287422CBF002702F0010772
:10594800002F3FF4C4AE08F1FF380027BFE68242BB
:1059580084BF584408F1FF38C8E7A24284BF09F160
:10596800FF395C44A6E79A4284BF0BF1FF3B1B1941
:1059780048E700BF2DE9F04F0C4683B08046164635
:1059880089461F4615468A46002B4BD18A425CD968
:10599800B2FA82F35BB1C3F1200001FA03FA28FAE4
:1059A80000F216FA03F508FA03F842EA0A0A2E0C7E
:1059B80050463146AFB2FFF723FC31464FEA184450
:1059C80081465046FFF74AFD07FB09F344EA014ABE
:1059D800534509D91AEB050A09F1FF3904D2534591
:1059E80084BF09F1FF39AA44C3EB0A0A314650467D
:1059F8001FFA88F8FFF704FC314604465046FFF7C3
:105A08002DFD07FB04F748EA0148474506D9013C44
:105A180018EB050802D2474588BF013C44EA09440F
:105A280000265CE08B4258D8B3FA83F6002E5BD18F
:105A38008B422CBF0022012285428CBF154642F0C2
:105A48000105002D49D0012449E022B91146012061
:105A5800FFF7D6FB0546B5FA85F6002E40F0BA806A
:105A6800641B2F0C1FFA85FA012639462046FFF7DA
:105A7800C7FB39464FEA184B81462046FFF7EEFC34
:105A88000AFB09F34BEA014B5B4509D91BEB050BF4
:105A980009F1FF3904D25B4584BF09F1FF39AB44F2
:105AA800C3EB0B0B394658461FFA88F8FFF7A8FBDB
:105AB800394604465846FFF7D1FC0AFB04FA48EA7F
:105AC8000148C24506D9013C18EB050802D2C24577
:105AD80088BF013C44EA094401E0002634463146C7
:105AE800204603B0BDE8F08FC6F12000B34032FA7B
:105AF80000F721FA00FB1F4314FA06F228FA00F116
:105B080058464FEA174A114300915146BBB20193D8
:105B1800FFF776FB5146B54081465846FFF79EFC95
:105B2800019C009804FB09F34FEA104C4CEA014B26
:105B38005B4505D91BEB070B09F1FF39C0F08E80D7
:105B4800C3EB0B0B51465846FFF75AFB5146044628
:105B58005846FFF783FC0198009A00FB04F31FFAEC
:105B680082FC4CEA0142934206D9013CD21903D285
:105B7800934201D9D219013C44EA0944A8B2D21A85
:105B88002D0C1FFA84FC230C00FB0CF700FB03FE12
:105B980005FB0CE105FB03F501EB17418E4588BFBA
:105BA80005F5803505EB1145AA4210D3BFB208FAB6
:105BB80006F607EB014214BF4FF0000E4FF0010E3E
:105BC80096422CBF00260EF00106002E87D0013C1D
:105BD800002684E7B540C6F1200124FA01F928FA25
:105BE80001F22F0CB4403946484622430092FFF791
:105BF80007FB39461FFA85FA83464846FFF72EFC0D
:105C0800009B1A0C0AFB0BF342EA0144A34203D996
:105C180064190BF1FF3B27D3E41A39462046FFF7F6
:105C2800EFFA394681462046FFF718FC00980AFB30
:105C380009F31FFA80FC4CEA0144A34208D964190D
:105C480009F1FF3904D2A34284BF09F1FF3964196D
:105C580008FA06F8E41A49EA0B4606E75B4584BFEA
:105C680009F1FF39BB446BE7A34284BF0BF1FF3B4B
:105C78006419D1E742F2FB1321F0004CC3F6E97333
:105C88009C45F0B5044687B00D4606460F461EDD16
:105C98004FF6FF73C7F6EF739C4505DD02460B46CA
:105CA800FAF7A2FD07B0F0BD02AA00F035F800F03F
:105CB800030001281DD0022810D008BB0123DDE90C
:105CC80002010093DDE9042300F036FFEAE7002231
:105CD80000230024009400F02FFFE3E70123DDE90F
:105CE80002010093DDE9042300F026FF01F10041E1
:105CF800D8E7DDE90201DDE9042300F019FAD1E76C
:105D0800DDE90201DDE9042300F012FA01F10041A6
:105D1800C8E700BF0000000042F2FB132DE9F04F76
:105D2800C3F6E97321F000468DB09E4282468B4649
:105D38000D46144640F39E804DF67B13C4F20203D1
:105D48009E4226DC0029DDA3D3E9002340F36181CC
:105D5800FAF74AFD42F2FB13C3F6F9739E428046F6
:105D6800894600F09C80D2A3D3E900230127FAF7E3
:105D78003BFD02460B46C4E9000140464946FAF796
:105D880033FDCBA3D3E90023FAF72EFDC4E90201C2
:105D980077E042F2FB13C4F239139E4240F39C8031
:105DA8004FF6FF73C7F6EF739E426EDC4FEA265834
:105DB8000246A8F582680DF11809A8F1060803271C
:105DC800A6EB0853CDE90223194609F10806FBF7AB
:105DD800D1F8083EFAF756FE02460B46CDE9060111
:105DE800DDE90201FAF700FD40F200030022C4F2E7
:105DF8007013FAF7ADFECDE90401FBF7BBF8FAF72B
:105E080041FE02460B46CDE90801DDE90401FAF737
:105E1800EBFC40F200030022C4F27013FAF798FE7C
:105E280000220023CDE90A01FFF77EFB48B1D6E93D
:105E3800020100220023013F083EFFF775FB0028FE
:105E4800F5D19D4E3B4648464246214601960226DC
:105E5800009600F095FA002D074612DA04F10803BF
:105E680062687F4202F1004262605A6802F10042B1
:105E78005A6006E00027C2E900AB00230022C4E90B
:105E8800022338460DB0BDE8F08F02460B46FAF7FC
:105E9800ABFC0027C4E90001C4E90201F1E77CA3D7
:105EA800D3E900230127FAF79FFC7BA3D3E900235A
:105EB80080468946FAF798FC02460B46C4E9000179
:105EC80040464946FAF790FC73A3D3E90023FAF752
:105ED8008BFCC4E90201D4E700F0E6FE70A3D3E925
:105EE800002380468946FAF733FE40F20003002279
:105EF800C3F6E073FAF77AFCFBF73CF80746FAF7C3
:105F0800C1FD69A3D3E90023CDE90201FAF720FE18
:105F180002460B4640464946FAF768FC64A3D3E9B3
:105F2800002380468946DDE90201FAF711FE1F2F9A
:105F380082468B4621DC47F288337A1EC0F600037E
:105F480053F82230B34218D052465B464046494681
:105F5800FAF74AFC02460B46C4E900234046494684
:105F6800FAF742FC5B465246FAF73EFC002D04F174
:105F78000803C4E9020184DA72E752465B464046E8
:105F88004946FAF731FC36150B46C1F30A51711A26
:105F980002461029C4E90023E0DD3DA3D3E900232C
:105FA800DDE90201FAF7D4FD82468B4652465B468C
:105FB80040464946FAF718FCCDE904014046DDE9B8
:105FC80004234946FAF710FC52465B46FAF70CFCE4
:105FD80031A3D3E9002380468946DDE90201FAF7B7
:105FE800B7FD42464B46FAF7FFFB82468B465246C0
:105FF8005B46DDE90401FAF7F7FB0B46C1F30A51EA
:10600800761A0246312EC4E900235BDCDDE90489F7
:10601800A4E7FAF7EBFB42F2FB13C3F6F9739E42CF
:106028008046894616D022A3D3E900234FF0FF37D4
:10603800FAF7DCFB02460B46C4E900014046494634
:10604800FAF7D2FB1AA3D3E90023FAF7CFFBC4E986
:10605800020116E70EA3D3E900234FF0FF37FAF742
:10606800C5FB0DA3D3E9002380468946FAF7BEFB9A
:1060780002460B46C4E9000140464946FAF7B4FB1C
:1060880005A3D3E90023FAF7B1FBC4E90201F8E656
:106098000000601A61B4D03D7370032E8A19A33BC7
:1060A80083C8C96D305FE43F00004054FB21F9BF4D
:1060B8003163621A61B4D03D08740008000040548E
:1060C800FB21F93F16A3D3E90023DDE90201FAF722
:1060D8003FFD82468B4652465B46DDE90401FAF7EE
:1060E80083FB8046894642464B46DDE90401FAF7C0
:1060F8007BFB52465B46FAF777FB0BA3D3E90023F9
:1061080082468B46DDE90201FAF722FD52465B46DC
:10611800FAF76AFB82468B4616E700BFAFF30080AA
:106128000000002E8A19A33BC14920259A837B3998
:106138002DE9F04F21F00046B6F1795F85B0804631
:10614800894692469B466FDAFAF714FF002800F05A
:10615800F98042464B4640464946FAF7F9FC7CA38B
:10616800D3E9002304460D46FAF7F2FC7AA3D3E9F3
:106178000023FAF73BFB22462B46FAF7E9FC78A303
:10618800D3E90023FAF730FB22462B46FAF7E0FC66
:1061980075A3D3E90023FAF729FB22462B46FAF721
:1061A800D7FC73A3D3E90023FAF71EFB22462B463C
:1061B800FAF7CEFC70A3D3E90023FAF717FB2246BF
:1061C8002B46FAF7C5FCCDE9000140F20003002296
:1061D80020462946C3F6E073FAF7BAFCDDE9002346
:1061E80006460F4620462946FAF7B2FC52465B4659
:1061F80004460D4640464946FAF7AAFC02460B46B5
:1062080020462946FAF7F0FA02460B463046394648
:10621800FAF7EAFA0B4640F200010246C3F6F071BB
:106228000020FAF7E1FA84E002460B46FAF790FC00
:1062380047A3D3E9002304460D46FAF789FC46A391
:10624800D3E90023FAF7D2FA22462B46FAF780FC64
:1062580043A3D3E90023FAF7C7FA22462B46FAF7F5
:1062680077FC41A3D3E90023FAF7C0FA22462B466C
:10627800FAF76EFC3EA3D3E90023FAF7B5FA2246F3
:106288002B46FAF765FC3CA3D3E90023FAF7AEFAEC
:106298002B462246FAF75CFC43F23233C3F6D3733B
:1062A8009E42CDE9000190DD40F20003C3F6E97398
:1062B8009E4241DD40F200070026C3F6D27740F245
:1062C800000132463B460020C3F6F071FAF78CFA1B
:1062D80040F200030022C3F6E073CDE90201204634
:1062E8002946FAF735FC32463B46FAF77DFADDE9EE
:1062F800002306460F4620462946FAF729FC52464F
:106308005B4604460D4640464946FAF721FC0246DC
:106318000B4620462946FAF767FA02460B463046EE
:106328003946FAF761FA02460B46DDE90201FAF747
:106338005BFA05B0BDE8F08FA6F5001300221646FB
:106348001F46BCE740F200010020C3F6F071F0E7F9
:10635800D43888BEE9FAA8BDC4B1B4BD9EEE213ECA
:10636800AD529C804F7E923E9015CB19A001FA3E0B
:106378007751C1166CC1563F4C5555555555A53FDB
:106388002DE9F04FADF51F7D144647F210558046B4
:10639800D01EA89AC0F600050A9118210C9355F84A
:1063A80022500B9500F0B0FD0C9B18220B9D013B71
:1063B800079320EAE0700E90C34302FB0342079C58
:1063C8002F1909921BD4041BA99862AEE71900EB98
:1063D800840509E028680435FAF754FBBC4204F147
:1063E8000104E6E802010AD0002CF3DA00200021BB
:1063F8000435BC42E6E8020104F10104F4D10B992A
:1064080000292FDB0C9B0DF1480BDDF81C900C9A32
:106418004FEAC30A8A180392DDF81CC0BCF1000FCA
:10642800C0F2AF8162A8002400EBC905002600274E
:1064380008EB040175E802230834D1E90001FAF7F2
:1064480087FB02460B4630463946FAF7CFF95445E2
:1064580006460F46ECD1039C09F10109EBE80267F7
:10646800A145D9D10B999EAC8AA80DF1480C4B1EB9
:1064780089468A00CDF804C004EB830410180F92F3
:10648800119410904FEAC90112AA8D18B9F1000FA2
:106498000391D5E9006730DD0024CB46C24640F2BF
:1064A80000030022C3F6706330463946FAF750FB02
:1064B800FAF760FDFAF7E6FA40F200030022CCF2A0
:1064C800701380468946FAF743FB32463B46FAF793
:1064D8008DF9FAF74FFD0DF50A7C75E90223494657
:1064E8004CF804004046FAF781F90434064601984E
:1064F8000F468542D3D1D946D04630463946099A07
:1065080000F06AFC00224FF07F5304460D46FAF76C
:106518001FFB00F0CDFB40F200030022CCF2200369
:10652800FAF716FB02460B4620462946FAF75EF9AB
:106538000D460446FAF71EFD8246FAF7A3FA02460C
:106548000B4620462946FAF74FF9099A002A0646CB
:106558000F4640F3F58009F1FF339EACC2F11801F4
:10656800C2F1170C04EB830353F8502C52FA01F0D4
:10657800824410FA01F1521A43F8502C42FA0CF5F1
:10658800002D3BDDB9F1000F0AF1010A40F3AA82A0
:1065980000234FEA89001C4607E019B10124C1F124
:1065A8008071D1500433834210D08AAAD158002C6C
:1065B800F3D04FF6FF720DF50A7CC0F2FF020124FA
:1065C800521A4CF8032004338342EED1099800286C
:1065D80011DD012800F0BD8002280CD109F1FF323D
:1065E8009EAB03EB820252F8503C23F07F4323F426
:1065F800400342F8503C022D00F083803046394673
:1066080000220023FEF790FF002800F0BF800B9CBB
:1066180009F1FF3084420EDC0DF50A7C00220CEBF8
:106628008903DDF840C053F8041D0A436345FAD1D5
:10663800002A40F03A82119850F8503C002B40F064
:106648004F820F998AAA5318012253F8081C013265
:10665800043B0029F9D04A440D9291454BDA0E9B30
:1066680012A8039903F1010B0C9C401804900C9894
:10667800CB44A99A09EB0403DDF834C0994602EB30
:106688008B0B4FEAC00A62AC844404EBC304CDF818
:1066980020C00394DBF80000FAF7F4F9079B039A8B
:1066A800002BC2E9000129DB62AC002604EBC90516
:1066B8000027002408EB040175E802230834D1E917
:1066C8000001FAF745FA02460B4630463946FAF712
:1066D8008DF8544506460F46ECD1039909F1010996
:1066E800089A0BF1040B0498083191450391E0E9ED
:1066F80002670490CED1DDF83490C3E60026002767
:10670800EBE740F2000132463B460020C3F6F07149
:10671800FAF76AF806460F46002C3FF46FAF40F2CE
:106728000001099A0020C3F6F07100F055FB0246FB
:106738000B4630463946FAF757F806460F465DE7E6
:1067480015D10DF51E7C0CEB890353F8545CED153F
:1067580016E709F1FF329EA901EB820252F8503C7C
:1067680023F07F4323F4000342F8503C43E740F210
:1067780000030022C3F6E073FEF7F4FE20B90025FB
:106788003CE70026002766E60225FBE60395CDF8E0
:106798001CA0002840F0AA81099B304639465A427D
:1067A80000F01AFB40F200030022C4F27013044602
:1067B8000D46FEF7D7FE002800F09B8140F200034B
:1067C8000022C3F6706320462946FAF7C1F90DF591
:1067D8001E7C0CEB8906FAF7CDFBFAF753F909F1A1
:1067E800010940F200030DF51E7C0022CCF2701363
:1067F8000CEB890782468B46FAF7AAF90B46024644
:1068080029462046F9F7F2FF099A18320992FAF751
:10681800B1FB594646F8500C5046FAF7ABFB47F81F
:10682800500C40F200010020099AC3F6F07100F004
:10683800D3FAB9F1000F06460F4658DB12AC8AAD01
:10684800A4F1080805EB890504EBC90455F8040907
:10685800FAF718F932463B46FAF77AF940F200039C
:106868000022C3F6706364E8020130463946FAF73D
:106878006FF9444506460F46E8D10B9F4FF00008D4
:10688800CDF81090002FC0F20981B8F1000FC0F2C6
:1068980005810DF1480C944E0CEBC9054FF0000A28
:1068A8004FF0000B002401E0444512DCD5E9002339
:1068B8000134D6E900010835FAF74AF908360246E4
:1068C8000B4650465946F9F791FFA74282468B4638
:1068D800EADA3AAC09F1FF3904EBC803B9F1FF3F32
:1068E80008F10108C3E900ABCCD1DDF81090A898F5
:1068F80003281CD8DFE810F0B7007D007D002300D6
:1069080000200146039A002A00F00681E36801F19D
:1069180000416268266803F10043A56802F100425D
:106928000A9C61612660A5606260E3602061DDF811
:106938001CC00CF007000DF51F7DBDE8F08FB9F104
:10694800000F3AACDCDD4FEAC9073B191E461D466D
:10695800D3E90001CDE90401DDE9042355E9020189
:10696800F9F744FF82468B46524655E902015B46D9
:10697800F9F73AFFDDE90423F9F738FFCDE904AB6D
:10698800C5E9000165E902ABA542E5D1B9F1010FFE
:10699800B6DD3F1909F1FF35D7E900AB04EBC505B2
:1069A800D5E9002350465946F9F720FF8046894625
:1069B8004246D5E900014B46F9F716FF02460B4659
:1069C80050465946F9F712FFC246CB46C5E90201BF
:1069D80065E80289A542E3D1002004F108050146D3
:1069E80076E8022380468946F9F700FFAE42F7D1E0
:1069F80088E7B9F1000FC0F28B803AAC002004EBB5
:106A0800C905A4F10806014675E8022382468B46AB
:106A1800F9F7ECFEB542F7D1039A002A43D001F109
:106A2800004C024606460A9867460B46C0E90067CE
:106A3800D4E90001F9F7D8FEB9F1000F09DD04EB3C
:106A4800C909F4E9022306460F46F9F7CFFE4C457B
:106A5800F7D1039A0AB101F100410A9C02460B469C
:106A6800C4E9022363E7B9F1000F4EDB3AAD002019
:106A780005EBC9040146083D74E8022306460F46A3
:106A8800F9F7B4FEAC42F7D1039A0AB101F100411B
:106A98000A9C02460B46C4E9002348E74FF0000A67
:106AA8004FF0000B15E78C46BBE70395CDF81CA00B
:106AB80083000DF51E7C03EB0C02099C52F8502C48
:106AC800183C0994FAB98AAA8146D318099A53F846
:106AD800041D09F1FF39183A0029F8D00992A0E6F7
:106AE8000122B8E5002471E52075000809F1FF309E
:106AF800DEE720469EAB294603EB8904FAF73AFA0B
:106B080044F8500C8DE681468BE600200146BBE731
:106B180000203AAC01467FE7D4E90267024630CC50
:106B28000B460A98C0E90423C0E90267C0E900459A
:106B3800FDE600BF000000002DE9F04F9B4621F064
:106B4800004385B0B3F1795F04460D46924603DAF7
:106B5800FAF710FA00286FD022462B46204629461D
:106B6800F9F7F6FF22462B4606460F46F9F7F0FFDF
:106B780041A3D3E900238046894630463946F9F7D0
:106B8800E7FF3FA3D3E90023F9F72EFE32463B4641
:106B9800F9F7DEFF3CA3D3E90023F9F727FE3246D5
:106BA8003B46F9F7D5FF3AA3D3E90023F9F71CFED2
:106BB80032463B46F9F7CCFF37A3D3E90023F9F770
:106BC80015FE0E9BCDE90001002B3AD040F20003E0
:106BD8000022C3F6E07350465946F9F7B9FFDDE9DC
:106BE8000023CDE9020140464946F9F7B1FF0246C4
:106BF8000B46DDE90201F9F7F7FD32463B46F9F7A6
:106C0800A7FF52465B46F9F7EFFD25A3D3E900231A
:106C180006460F4640464946F9F79AFF02460B4694
:106C280030463946F9F7E2FD02460B46204629462A
:106C3800F9F7DAFD04460D462046294605B0BDE8B9
:106C4800F08F02460B4630463946F9F781FF14A308
:106C5800D3E90023F9F7C8FD42464B46F9F778FF18
:106C680002460B4620462946F9F7C0FD04460D4664
:106C7800E2E700BFAFF300807CD5CF5A3AD9E53DB3
:106C8800EB9C2B8AE6E55A3E7DFEB157E31DC73ED5
:106C9800D561C119A0012A3FA6F810111111813F31
:106CA800495555555555C53F21F00043194670477C
:106CB8002DE9F047C1F30A54A4F57E740246073C57
:106CC8000B46132C06460F460D468A46804621DCA5
:106CD800002C40DB4FF6FF7CC0F20F0C4CFA04F995
:106CE80009EA0105054311D039A3D3E90023F9F7CF
:106CF8007DFD00220023FEF73FFC00283CD0002F3A
:106D08005DDB2AEA090A002553462A461046194639
:106D1800BDE8F087332C07DDB4F5806FF6D1F9F7BD
:106D280065FD02460B46F1E74FF0FF35A4F1140C60
:106D380025FA0CF50542E9D025A3D3E90023F9F794
:106D480055FD00220023FEF717FCA8B1002F1BDB1E
:106D580026EA05050AE01EA3D3E90023F9F746FD54
:106D680000220023FEF708FC48B9354653462A4658
:106D780010461946BDE8F0873546BA46F6E7002FB3
:106D880010DB0025AA46F1E7142C06D00126C4F131
:106D98003404A64016EB0806DAD30AF1010A26EAFB
:106DA8000505E3E727F0004540F2000A3543CBF636
:106DB800F07A002D08BFBA4618BF0025D6E74FF471
:106DC800801353FA04F407EB040A9AE7AFF3008040
:106DD8009C7500883CE4377EC1F30A532DE9D04303
:106DE800144606460F46804689460A46002B2FD190
:106DF80021F00042024327D040F200030022C4F2EF
:106E08005033F9F7A5FE43F6B043CFF6FF739C4223
:106E180006460F46804689463ADBC1F30A530A46BE
:106E2800363B40F2FE711B198B421ADD32463B4657
:106E38002BA1D1E9000100F05BF829A3D3E90023D5
:106E4800F9F786FE06460F4630463946BDE8D08338
:106E580040F2FF7C634526D01B1940F2FE718B423D
:106E6800E4DC002BC2BF22F0FE4222F4700242EAA8
:106E78000357E9DC13F1350F1FDA4CF250339C420B
:106E8800D4DC32463B4618A1D1E9000100F030F8C5
:106E980015A3D3E90023F9F75BFE06460F463046F3
:106EA8003946BDE8D08302460B46F9F79FFC0646F3
:106EB8000F4630463946BDE8D083363322F0FE42CD
:106EC80022F47002304642EA035740F20003394682
:106ED8000022C3F69043F9F73BFE06460F46B3E798
:106EE8009C7500883CE4377E59F3F8C21F6EA501F3
:106EF80003F0004321F0004230B40D46044643EA53
:106F0800020130BC704700BF002900F03E8180EAD2
:106F1800010C48BF49424A1E00F01F81031C48BFAC
:106F280043428B4240F21E81114200F02381B3FAA2
:106F380083F2B1FA81F0A0EB0202C2F11F0204A0B1
:106F480000EB02124FF00000974600BFAFF300803D
:106F5800B3EBC17F00BF40EB000028BFA3EBC173B8
:106F6800B3EB817F00BF40EB000028BFA3EB817328
:106F7800B3EB417F00BF40EB000028BFA3EB417398
:106F8800B3EB017F00BF40EB000028BFA3EB017308
:106F9800B3EBC16F00BF40EB000028BFA3EBC16398
:106FA800B3EB816F00BF40EB000028BFA3EB816308
:106FB800B3EB416F00BF40EB000028BFA3EB416378
:106FC800B3EB016F00BF40EB000028BFA3EB0163E8
:106FD800B3EBC15F00BF40EB000028BFA3EBC15378
:106FE800B3EB815F00BF40EB000028BFA3EB8153E8
:106FF800B3EB415F00BF40EB000028BFA3EB415358
:10700800B3EB015F00BF40EB000028BFA3EB0153C7
:10701800B3EBC14F00BF40EB000028BFA3EBC14357
:10702800B3EB814F00BF40EB000028BFA3EB8143C7
:10703800B3EB414F00BF40EB000028BFA3EB414337
:10704800B3EB014F00BF40EB000028BFA3EB0143A7
:10705800B3EBC13F00BF40EB000028BFA3EBC13337
:10706800B3EB813F00BF40EB000028BFA3EB8133A7
:10707800B3EB413F00BF40EB000028BFA3EB413317
:10708800B3EB013F00BF40EB000028BFA3EB013387
:10709800B3EBC12F00BF40EB000028BFA3EBC12317
:1070A800B3EB812F00BF40EB000028BFA3EB812387
:1070B800B3EB412F00BF40EB000028BFA3EB4123F7
:1070C800B3EB012F00BF40EB000028BFA3EB012367
:1070D800B3EBC11F00BF40EB000028BFA3EBC113F7
:1070E800B3EB811F00BF40EB000028BFA3EB811367
:1070F800B3EB411F00BF40EB000028BFA3EB4113D7
:10710800B3EB011F00BF40EB000028BFA3EB011346
:10711800B3EBC10F00BF40EB000028BFA3EBC103D6
:10712800B3EB810F00BF40EB000028BFA3EB810346
:10713800B3EB410F00BF40EB000028BFA3EB4103B6
:10714800B3EB010F00BF40EB000028BFA3EB010326
:10715800BCF1000F48BF404270479CEA000F48BF8F
:107168004042704738BF002004BF4FEAEC7040F03F
:1071780001007047B1FA81F2C2F11F02BCF1000FA1
:1071880023FA02F048BF404270470028C8BF6FF09A
:107198000040B8BF4FF00040FEF76EB90029F4D0A8
:1071A8002DE90340FFF7B3FEBDE8064002FB00F3FC
:1071B800A1EB0301704700BF002103E00A4B5B58B5
:1071C8004350043109480A4B42189A42F6D3094AF7
:1071D80002E0002342F8043B074B9A42F9D3F9F73F
:1071E80017F8F9F7D5F970471C7600080000002059
:1071F800040500200405002044050020FEE70000E7
:107208002020202020202020202020202020202076
:107218003030303030303030303030303030303066
:10722800E8750008E47500089C7500089C7500085E
:107238009C7500089C7500089C7500089C750008E2
:107248009C7500089C7500089C750008FFFFFFFFEF
:10725800FFFFFFFF00000000000000000000F03FFB
:107268000000000000002440000000000000594019
:107278000000000000408F40000000000088C3406C
:1072880000000000006AF8400000000080842E41E1
:1072980000000000D01263410000000084D797412D
:1072A8000000000065CDCD41000000205FA0024233
:1072B800000000E876483742000000A2941A6D42A8
:1072C800000040E59C30A2420000901EC4BCD6429B
:1072D80000003426F56B0C430080E03779C3414346
:1072E80000A0D8855734764300C84E676DC1AB43BC
:1072F800003D9160E458E143408CB5781DAF1544DA
:1073080050EFE2D6E41A4B4492D54D06CFF08044B4
:10731800F64AE1C7022DB544B49DD9794378EA44C9
:1073280005000000190000007D00000000000000BA
:107338000080E03779C34143176E05B5B5B8934669
:10734800F5F93FE9034F384D321D30F94877825A35
:107358003CBF737FDD4F1575BC89D897B2D29C3C72
:1073680033A7A8D523F649393DA7F444FD0FA53224
:107378009D978CCF08BA5B25436FAC642806C80A72
:10738800FB21F93FFB2109407CD91240FB21194020
:107398007A6A1F407CD92240BBFD2540FB21294049
:1073A8003A462C407A6A2F405C4731407CD93240BB
:1073B8009C6B3440BBFD3540DB8F3740FB213940A7
:1073C8001BB43A403A463C405AD83D407A6A3F405E
:1073D8004C7E40405C4741406C1042407CD9424062
:1073E8008CA243409C6B4440AC344540BBFD4540B7
:1073F800CBC64640DB8F4740EB584840FB2149400D
:1074080083F9A200444E6E00FC291500D1572700CD
:10741800DD34F50062DBC0003C99950041904300E3
:107428006351FE00BBDEAB00B761C5003A6E2400B5
:10743800D24D42004906E00009EA2E001C92D10014
:10744800EB1DFE0029B11C00E83EA700F5358200BF
:1074580044BB2E009CE98400B4267000417E5F0086
:10746800D6913900538339009CF439008B5F84002E
:1074780028F9BD00F81F3B00DEFF97000F980500B4
:10748800112FEF000A5A8B006D1F6D00CF7E36005A
:1074980009CB2700464FB7009E663F002DEA5F00E4
:1074A800BA277500E5EBC7003D7BF100F739070007
:1074B80092528A00FB6BEA001FB15F00085D8D00E5
:1074C800300356007BFC4600F0AB6B0020BCCF00BD
:1074D80036F49A00E3A91D005E619100081BE600DE
:1074E80085996500A0145F008D40680080D8FF0072
:1074F80027734D0006063100CA561500C9A8730047
:107508007BE260006B8CC0000200000003000000FA
:10751800040000000600000000000040FB21F93FC5
:10752800000000002D44743E000000809846F83C9E
:107538000000006051CC783B00000080831BF039CC
:107548000000004020257A38000000802282E336BF
:10755800000000001DF369350A5465737420666CD9
:107568006F61742073696E75730D0A00252E3230B1
:107578006C6609252E32306C660D0A00646F6E65E4
:107588000A0D00003031323334353637383941424C
:107598004344454600000000494E4600696E6600B7
:1075A8004E414E006E616E0030313233343536371D
:1075B800383961626364656600000000286E756C86
:1075C8006C29000030000000496E66696E697479A4
:1075D800000000004E614E00430000002E00000035
:1075E80049534F2D383835392D310000F8B500BFD3
:1075F800F8BC08BC9E467047F8B500BFF8BC08BC8C
:047608009E467047E3
:08760C000CE0FF7F010000000B
:04761400FD0100086C
:04761800E90100087C
:10761C00040000200000000000000000000000003A
:10762C00000000000000000000000000000000004E
:10763C0000000000E07500080000000000000000E1
:10764C00000000000000000000000000000000002E
:10765C00000000000000000000000000000000001E
:10766C00000000000000000000000000000000000E
:10767C0000000000000000000000000000000000FE
:10768C0000000000000000000000000000000000EE
:10769C0000000000000000000000000000000000DE
:1076AC0000000000000000000000000000000000CE
:1076BC0000000000000000000000000000000000BE
:1076CC0000000000000000000000000000000000AE
:1076DC00000000000000000000000000000000009E
:1076EC00000000000000000000000000000000008E
:1076FC00000000000000000000000000000000007E
:10770C00000000000000000000000000F400002059
:10771C00F4000020FC000020FC00002004010020EC
:10772C00040100200C0100200C0100201401002099
:10773C00140100201C0100201C0100202401002049
:10774C00240100202C0100202C01002034010020F9
:10775C00340100203C0100203C01002044010020A9
:10776C00440100204C0100204C0100205401002059
:10777C00540100205C0100205C0100206401002009
:10778C00640100206C0100206C01002074010020B9
:10779C00740100207C0100207C0100208401002069
:1077AC00840100208C0100208C0100209401002019
:1077BC00940100209C0100209C010020A4010020C9
:1077CC00A4010020AC010020AC010020B401002079
:1077DC00B4010020BC010020BC010020C401002029
:1077EC00C4010020CC010020CC010020D4010020D9
:1077FC00D4010020DC010020DC010020E401002089
:10780C00E4010020EC010020EC010020F401002038
:10781C00F4010020FC010020FC01002004020020E7
:10782C00040200200C0200200C0200201402002094
:10783C00140200201C0200201C0200202402002044
:10784C00240200202C0200202C02002034020020F4
:10785C00340200203C0200203C02002044020020A4
:10786C00440200204C0200204C0200205402002054
:10787C00540200205C0200205C0200206402002004
:10788C00640200206C0200206C02002074020020B4
:10789C00740200207C0200207C0200208402002064
:1078AC00840200208C0200208C0200209402002014
:1078BC00940200209C0200209C020020A4020020C4
:1078CC00A4020020AC020020AC020020B402002074
:1078DC00B4020020BC020020BC020020C402002024
:1078EC00C4020020CC020020CC020020D4020020D4
:1078FC00D4020020DC020020DC020020E402002084
:10790C00E4020020EC020020EC020020F402002033
:10791C00F4020020FC020020FC02002004030020E2
:10792C00040300200C0300200C030020140300208F
:10793C00140300201C0300201C030020240300203F
:10794C00240300202C0300202C03002034030020EF
:10795C00340300203C0300203C030020440300209F
:10796C00440300204C0300204C030020540300204F
:10797C00540300205C0300205C03002064030020FF
:10798C00640300206C0300206C03002074030020AF
:10799C00740300207C0300207C030020840300205F
:1079AC00840300208C0300208C030020940300200F
:1079BC00940300209C0300209C030020A4030020BF
:1079CC00A4030020AC030020AC030020B40300206F
:1079DC00B4030020BC030020BC030020C40300201F
:1079EC00C4030020CC030020CC030020D4030020CF
:1079FC00D4030020DC030020DC030020E40300207F
:107A0C00E4030020EC030020EC030020F40300202E
:107A1C00F4030020FC030020FC03002004040020DD
:107A2C00040400200C0400200C040020140400208A
:107A3C00140400201C0400201C040020240400203A
:107A4C00240400202C0400202C04002034040020EA
:107A5C00340400203C0400203C040020440400209A
:107A6C00440400204C0400204C040020540400204A
:107A7C00540400205C0400205C04002064040020FA
:107A8C00640400206C0400206C04002074040020AA
:107A9C00740400207C0400207C040020840400205A
:107AAC00840400208C0400208C040020940400200A
:107ABC00940400209C0400209C040020A4040020BA
:107ACC00A4040020AC040020AC040020B40400206A
:107ADC00B4040020BC040020BC040020C40400201A
:107AEC00C4040020CC040020CC040020D4040020CA
:107AFC00D4040020DC040020DC040020E40400207A
:107B0C00E4040020EC040020EC040020FFFFFFFF45
:047B1C000000020063
:04000005080071C1BD
:00000001FF
